:020000020000FC
:100000000C94D54D18951895189518951895189520
:100010001895189518951895189518951895189578
:100020001895189518951895189518951895189568
:100030001895189518951895189518950C941F30C3
:1000400018951895189518950C9450491895189569
:100050001895189518951895189518951895189538
:100060001895189518951895189518951895189528
:1000700018951895189518950C942A49189518955F
:100080001895189518951895189518950D0A20002B
:100090000D0A0A205B434D2D352056657273696F3A
:1000A0006E20312E31355D000D0A20546F737320A0
:1000B0004D6F64650D0A000D0A202D3E5B44796E7C
:1000C000616D6978656C5D3A000D0A203C2D5B44DA
:1000D000796E616D6978656C5D3A000D0A203C2D82
:1000E0003E50433A00203C2D3E44796E616D697864
:1000F000656C3A000D0A2041726520796F75207396
:10010000757265203F28792F4E29000D0A205573FE
:10011000616765203A20476F205B506F736974698F
:100120006F6E20416E676C6528307830307E307895
:10013000336666295D000D0A20416C6C2044796E9F
:10014000616D6978656C27732049442077696C6C10
:100150002062652073657420746F20002E20417228
:100160006520796F7520737572653F28592F4E2968
:10017000000D0A204572726F72315B436865636BD4
:100180002044796E616D6978656C2056657273697B
:100190006F6E206973206D6F7265207468616E20C8
:1001A000335D000D0A2042284265666F7265292C76
:1001B0004E284E657874292C512851756974290090
:1001C0000D0A203438354D6F6E69746F72205B4CA8
:1001D000462C43522061726520616464656420612D
:1001E000742070617573652074696D655D0D0A001A
:1001F0000D0A204E6F20446174615B61742042726D
:100200006F61646361737420494420307846455DB2
:10021000000D0A204E6F20446174612843686563B5
:100220006B2049442C204F7065726174696E6720A1
:100230004D6F64652C20426175642072617465297C
:1002400000204C454E3A000D0A204C454420426C9B
:10025000696E6B2049443A002044796E616D69787B
:10026000656C7320466F756E642E000D0A204C4538
:100270004420426C696E6B2049443A000D20466F61
:10028000756E642120424155445F5245473A002C27
:100290002049443A000D0A20426175642052656786
:1002A000206973206368616E67656420746F200045
:1002B000425053000D0A2049443A30202D20000DB1
:1002C0000A2044656C61793A000D0A20546F7271FE
:1002D000756520456E61626C65000D0A204D6F7674
:1002E000652030203C2D3E203078336666000D0AB4
:1002F00020416E79204B657920746F20436F6E74B6
:10030000696E75652E2E2E000D0A205B45455052F4
:100310004F4D20415245415D0D0A204D4F44454C03
:100320005F4E554D4245525F4C202020202020201A
:1003300020285229205B000D0A204D4F44454C5F78
:100340004E554D4245525F4820202020202020203D
:10035000285229205B000D0A2056455253494F4E22
:100360002020202020202020202020202020202885
:100370005229205B000D0A20494420202020202003
:100380002020202020202020202020202028522F24
:1003900057295B000D0A20424155445F52415445A4
:1003A00020202020202020202020202028522F57CD
:1003B000295B000D0A2052455455524E5F44454C6E
:1003C00041595F54494D452020202028522F57295C
:1003D0005B000D0A2043575F414E474C455F4C4937
:1003E0004D49545F4C202020202028522F57295B54
:1003F000000D0A2043575F414E474C455F4C494D25
:1004000049545F48202020202028522F57295B0084
:100410000D0A204343575F414E474C455F4C494DC1
:1004200049545F4C2020202028522F57295B000D73
:100430000A204343575F414E474C455F4C494D4965
:10044000545F482020202028522F57295B000D0A96
:10045000202852455345525645442920202020202B
:1004600020202020202028522F57295B000D0A2011
:100470004C494D49545F54454D5045524154555295
:10048000452020202028522F57295B000D0A2044A8
:100490004F574E5F4C494D49545F564F4C5441475E
:1004A0004520202028522F57295B000D0A20555047
:1004B0005F4C494D49545F564F4C544147452020AD
:1004C00020202028522F57295B000D0A204D41582B
:1004D0005F544F525155455F4C2020202020202052
:1004E000202028522F57295B000D0A204D41585FCC
:1004F000544F525155455F48202020202020202075
:100500002028522F57295B000D0A2052455455527E
:100510004E5F4C4556454C20202020202020202096
:1005200028522F57295B000D0A20414C41524D5F44
:100530004C4544202020202020202020202020283E
:10054000522F57295B000D0A20414C41524D5F53F9
:10055000485554444F574E20202020202020285218
:100560002F57295B000D0A20285245534552564506
:100570004429202020202020202020202028522F05
:1005800057295B000D0A20444F574E5F43414C49A9
:1005900042524154494F4E5F4C20202028522F5741
:1005A000295B000D0A20444F574E5F43414C49429E
:1005B000524154494F4E5F4820202028522F57293E
:1005C0005B000D0A2055505F43414C494252415453
:1005D000494F4E5F4C202020202028522F57295B66
:1005E000000D0A2055505F43414C49425241544945
:1005F0004F4E5F48202020202028522F57295B0093
:100600000D0A205B52414D20415245415D0D0A20AB
:10061000544F525155455F454E41424C4520202094
:10062000202020202028522F57295B000D0A204C23
:100630004544202020202020202020202020202071
:100640002020202028522F57295B000D0A204357D5
:100650005F434F4D504C49414E43455F4D415247DA
:10066000494E2028522F57295B000D0A204343573B
:100670005F434F4D504C49414E43455F4D415247BA
:10068000494E28522F57295B000D0A2043575F43DC
:100690004F4D504C49414E43455F534C4F504520C0
:1006A0002028522F57295B000D0A204343575F43F0
:1006B0004F4D504C49414E43455F534C4F504520A0
:1006C00028522F57295B000D0A20474F414C5F509D
:1006D0004F534954494F4E5F4C2020202020202862
:1006E000522F57295B000D0A20474F414C5F504F56
:1006F000534954494F4E5F48202020202020285243
:100700002F57295B000D0A204D4F56494E475F5326
:10071000504545445F4C2020202020202028522F87
:1007200057295B000D0A204D4F56494E475F5350E5
:100730004545445F482020202020202028522F5764
:10074000295B000D0A20544F525155455F4C494DCD
:1007500049545F4C2020202020202028522F572948
:100760005B000D0A20544F525155455F4C494D498D
:10077000545F482020202020202028522F57295B1A
:10078000000D0A2050524553454E545F504F534977
:1007900054494F4E5F4C20202020285229205B00D6
:1007A0000D0A2050524553454E545F504F53495403
:1007B000494F4E5F4820202020285229205B000D01
:1007C0000A2050524553454E545F53504545445FAF
:1007D0004C20202020202020285229205B000D0AB8
:1007E0002050524553454E545F53504545445F4851
:1007F00020202020202020285229205B000D0A20C4
:1008000050524553454E545F4C4F41445F4C20205D
:10081000202020202020285229205B000D0A205073
:10082000524553454E545F4C4F41445F4820202071
:100830002020202020285229205B000D0A20505221
:100840004553454E545F564F4C5441474520202058
:1008500020202020285229205B000D0A20505245DC
:1008600053454E545F54454D5045524154555245A1
:10087000202020285229205B000D0A20524547499C
:100880005354455245445F494E53545255432E20CC
:100890002028522F57295B000D0A205245534552FC
:1008A0005645442850415553455F54494D452920EC
:1008B00028522F57295B000D0A204D4F56494E47AD
:1008C0002020202020202020202020202020202028
:1008D000285229205B000D0A204C4F434B2020203A
:1008E00020202020202020202020202020202852CE
:1008F0002F57295B000D0A2050554E43485F4C206E
:100900002020202020202020202020202028522F9E
:1009100057295B000D0A2050554E43485F48202060
:1009200020202020202020202020202028522F5747
:10093000295B000D0A0A2044554D50284429203ACD
:100940002044756D7020636F6E74726F6C207461DB
:10095000626C652E000D0A204944205B49445F4EBD
:10096000554D5D203A20536574204944206F662020
:1009700064796E616D6978656C2E000D0A204349BB
:1009800044205B49445F4E554D5D203A20436861E9
:100990006E676520436F6E74726F6C2049442E0041
:1009A0000D0A2052454144205B414444525D5B4C5A
:1009B000454E5D203A205265616420646174612E69
:1009C0002065782952656164203130203220285218
:1009D0006561642066726F6D20307831302C206C38
:1009E000656E677468203229000D0A2057524954F9
:1009F00045205B414444525D5B44415441315D2E8E
:100A00002E203A20577269746520646174612E202B
:100A100065782957726974652031342C3120285744
:100A20007269746520312061742030783134290076
:100A30000D0A205245475F5752205B414444525DA6
:100A40005B44415441315D2E2E203A205265676946
:100A50007374657220777269746520696E7374753A
:100A6000726374696F6E000D0A20414354494F4E02
:100A7000203A20416374696F6E205245475F575298
:100A800020696E737472756374696F6E000D0A204D
:100A9000476F205B504F534954494F4E5D5B535055
:100AA0004545445D3A20476F746F20746865207037
:100AB0006F736974696F6E207769746820746865F4
:100AC0002073706565642E000D0A20484558205B30
:100AD0004E554D5D5B4E554D5D2E2E2E203A2054C9
:100AE00072616E736D6974652072617720646174E0
:100AF000612E2065782948657820464620464620A4
:100B00003031203033000D0A205245534554203AED
:100B10002044796E616D6978656C205265736574E7
:100B20002E000D0A2050494E47205B4E554D5D3A30
:100B3000206578292050696E67204E554D20494424
:100B40002064796E616D6978656C2E000D0A205302
:100B50005752205B414444525D5B4C454E5D5B49BE
:100B6000445D5B444154415D2E2E2E5B49445D5BE8
:100B7000444154415D2E2E2E203A2053796E63203D
:100B800057726974652E000D0A205343414E205B55
:100B90004E554D5D203A205343414E206C696E6B9B
:100BA00065642064796E616D6978656C20696E207A
:100BB000307E4E554D20696E2063757272656E747D
:100BC000206261756420726174652E000D0A204CEC
:100BD0004544205B4E554D5D203A20426C696E6B5A
:100BE000204C4544206F66204E554D2049442E2010
:100BF0002742272C274E2720666F72204944206306
:100C000068616E67652E2027512720666F7220511C
:100C10007569742E000D0A2042415544205B4E55E3
:100C20004D5D203A205365742062617564207261C5
:100C300074652020657829204241554420323228AD
:100C40003537363030425053292C2042415544200C
:100C50003128314D42505329000D0A20534541524D
:100C60004348203A205365617263682049442061FB
:100C70006E64206261756472617465206F662061C4
:100C80006C6C206C696E6B65642064796E616D6953
:100C900078656C732E000D0A2055706461746520B0
:100CA0005B53544152545F49445D205B454E445F61
:100CB00049445D203A2044796E616D6978656C2005
:100CC0006669726D77617265207570646174652EF6
:100CD0002873797374656D2075736572206F6E6CFF
:100CE0007929000D0A0A2020202020202020436F8F
:100CF0007079726967687420524F424F544953208B
:100D0000434F2E2C4C54442E0D0A005B496E7661E5
:100D10006C6964205061676520526561643A000D1A
:100D20000A205B4572723A5278442054696D656FAF
:100D300075745D000D0A205B4572723A57726F6ED2
:100D400067204865616465725D000D0A205B45722D
:100D5000723A5478494420213D20527849445D003C
:100D60000D0A205B4572723A57726F6E67204C65B0
:100D70006E6774685D000D0A205B4572723A5772A7
:100D80006F6E6720436865636B53756D5D000D0A78
:100D900020555044415445205B53544152542049FE
:100DA000445D205B454E442049445D005D3A000DA2
:100DB0000A2049443A00205374616E6462792E001F
:100DC0002057726974696E672E2E00205375636315
:100DD0006573732E00204572726F722E000D0A200B
:100DE0004572722049443A002042616420436F6D8D
:100DF0006D616E64005B457869745D005B53544FB0
:100E0000505D000D0A204D4F54494F4E20504C412B
:100E10005920504147452020202028522F57290093
:100E20000D0A204F4E20504C4159494E47204D4FFE
:100E300054494F4E2020202028522920000D0A20FE
:100E4000545820574952454C455353205041434B29
:100E50004554202028522F5729000D0A205258208F
:100E6000574952454C455353205041434B4554201C
:100E7000202028522920000D0A204E45572050419D
:100E8000434B455420415252495645442020202886
:100E9000522920000D0A20415558204C454420205D
:100EA000202020202020202020202028522F5729B9
:100EB000000D0A20425554544F4E282D532D552DC8
:100EC000442D4C2D522920202028522920000D0A83
:100ED0002054494D4552283132356D5365632045C4
:100EE000616368292028522F5729000D0A205A498A
:100EF0004742454520494420202020202020202012
:100F0000202028522F5729000D0A20524F424F54BB
:100F1000204944202020202020202020202020287C
:100F2000522F5729000D44796E616D6978656C20E8
:100F300020302830783030295B202020205D000DC3
:100F40000A44796E616D6978656C202031283078AB
:100F50003031295B202020205D0020506167654EE4
:100F6000756D6265723A000D0A44796E616D69783B
:100F7000656C2020322830783032295B20202020F8
:100F80005D0020416464723A000D0A44796E616D1F
:100F90006978656C2020332830783033295B202035
:100FA00020205D00202852657365727665642920D3
:100FB0003A000D0A44796E616D6978656C202034C1
:100FC0002830783034295B202020205D002020202C
:100FD000506C6179436F756E743A000D0A44796EF6
:100FE000616D6978656C2020352830783035295B53
:100FF000202020205D00202852657365727665648C
:1010000029203A000D0A44796E616D6978656C207B
:1010100020362830783036295B202020205D0020C3
:1010200028526573657276656429203A000D0A447A
:10103000796E616D6978656C20203728307830379B
:10104000295B202020205D00202852657365727680
:10105000656429203A000D0A44796E616D697865EE
:101060006C2020382830783038295B202020205D03
:10107000002028526573657276656429203A000D58
:101080000A44796E616D6978656C20203928307862
:101090003039295B202020205D002020205061670E
:1010A0006520537465703A000D0A44796E616D696C
:1010B00078656C2031302830783041295B20202041
:1010C000205D0020436F6E74726F6C436F64653AED
:1010D000000D0A44796E616D6978656C20313128A4
:1010E00030783042295B202020205D002020506194
:1010F00067652053706565643A000D0A44796E6136
:101100006D6978656C2031322830783043295B2056
:101110002020205D0020202044584C205365747509
:10112000703A000D0A44796E616D6978656C203102
:10113000332830783044295B202020205D00202097
:10114000416363656C2054696D653A000D0A44790A
:101150006E616D6978656C203134283078304529AE
:101160005B202020205D004C696E6B20746F204E48
:101170006578743A000D0A44796E616D6978656C22
:101180002031352830783046295B202020205D0032
:101190004C696E6B20746F20457869743A000D0AB3
:1011A00044796E616D6978656C203136283078310C
:1011B00030295B202020205D0028526573657276FF
:1011C00065645031293A000D0A44796E616D697881
:1011D000656C2031372830783131295B2020202080
:1011E0005D002852657365727665645231293A0054
:1011F0000D0A44796E616D6978656C20313828304C
:10120000783132295B202020205D002852657365EB
:10121000727665645032293A000D0A44796E616D28
:101220006978656C2031392830783133295B20208A
:1012300020205D00285265736572766564523229FC
:101240003A000D0A44796E616D6978656C20323020
:101250002830783134295B202020205D000D0A449D
:10126000796E616D6978656C20323128307831355E
:10127000295B202020205D000D0A44796E616D6994
:1012800078656C2032322830783136295B20202076
:10129000205D000D0A44796E616D6978656C2032BD
:1012A000332830783137295B202020205D000D0A5B
:1012B00044796E616D6978656C20323428307831FC
:1012C00038295B202020205D000D0A44796E616D75
:1012D0006978656C2032352830783139295B2020D7
:1012E00020205D000D0A44796E616D6978656C207F
:1012F00032362830783161295B202020205D000DB6
:101300000A44796E616D6978656C203237283078CF
:101310003162295B202020205D000D0A44796E6136
:101320006D6978656C2032382830783163295B200C
:101330002020205D000D0A44796E616D6978656C2E
:101340002032392830783164295B202020205D004C
:101350000D0A44796E616D6978656C2033302830F0
:10136000783165295B202020205D000D0A20202097
:10137000506175736554696D652020202020202000
:101380005B2020205D000D0A2020205370656564DD
:101390002020202020202020202020000D0A202096
:1013A0002054696D6528207820372E386D53656389
:1013B00029005B2020205D202020202020202020CC
:1013C000202020202020202020202020202020201D
:1013D00020202020202020202020205B583A2D2D66
:1013E0002C593A2D2D2C413A2D2D2D2D5D000D0A15
:1013F00020202020202020202020202020202020ED
:101400002020205354503720205354503020535420
:1014100050312053545032205354503320535450A1
:101420003420535450352053545036202020204728
:101430006F20537465703A2020202020000D0A2070
:10144000202020202020202020202020202020209C
:1014500020202020202020204D53545220534C4146
:1014600056204F465354202020202020202020208A
:101470002020202020202020202020202020476FF6
:1014800020537465703A2020202020000D0A5D2032
:101490005F2020202020202020202020202020200D
:1014A000202020202020202020202020202020203C
:1014B000202020202020202020202020202020202C
:1014C000202020202020202020202020202020201C
:1014D0002020202020202020202000204172652074
:1014E000796F7520737572653F5B792F4E5D0020B3
:1014F000496E76616C696420506167650020496EB1
:1015000076616C696420506172616D65746572000A
:10151000204F66667365742055706461746564005D
:10152000204F7574206F662052616E676500204FF2
:101530004B000D0A20202020202020202D434D3A52
:101540002052503D2850617261302C4F502C506118
:1015500072613129204C4B205253205B414444524C
:101560005D2020000D0A20427265616B20617420AD
:10157000000D0A204552524F523A00494620202081
:10158000202000454C534520494600454C534520FA
:10159000202000616E642F6F7220004A554D50204C
:1015A0002020004C4F414420202000434F4D5055F7
:1015B0005445005354415254202000454E442020AD
:1015C00020200043414C4C202020005245545552CD
:1015D0004E20004E554C4C202020000D0A2048453E
:1015E000584120444953504C4159204D4F444500E7
:1015F0000D0A20444543494D414C20444953504C29
:101600004159204D4F44450003404C464D4840450C
:101610004A230102030A222121217D7D7D7D7D7DDA
:101620007D7D7D7D7D7D7D7D7D797673716E6C693F
:1016300067656361605E5C5B595857555453515000
:101640004F4E4D4C4B4A4948474645444342424120
:10165000403F3F3E3D3C3C3B3A39393837373636E0
:10166000353434333332313130302F2F2E2D2D2C71
:101670002C2B2B2A2A2929282827272626252525E9
:1016800024242323222221212020201F1F1E1E1D4F
:101690001D1D1C1C1B1B1A1A1A19191818181717AC
:1016A0001616161515141414131312121211111004
:1016B00010100F0F0E0E0E0D0D0C0C0C0B0B0A0A5A
:1016C00009090908080707070606050504040403B5
:1016D0000302020101010000000000000000000000
:1016E00000000000000000000000000000000000FA
:1016F00000000000000000000000000000000000EA
:1017000000000000000000000000000000000000D9
:1017100000000000000000000000000000010101C6
:1017200002000200010101010200010101010200A9
:101730000200010101010101020002000200020099
:101740000200020001010101010102000101020089
:10175000020000000001010101010000010101017E
:101760000100010101010101000001010000000070
:101770000000010000000101020001010000010160
:101780000101020002000101682FA901812F00233D
:10179000B9F40FE003BF00E002BF09E01DE30E94BF
:1017A0002D4E10E0003021E0120710F000E009C0DB
:1017B00001BF082F00FB07B701F907BF01E001C017
:1017C00000E0862F089500E00093610002B901BB9C
:1017D00004BB07BB0ABB00E00093650000936200F6
:1017E00003B902BB05BB08BB00B50B7F00BD00B54C
:1017F0000B7F00BD00E00093610002B901BB04BB98
:1018000007BB0ABB00E0009365000093620003B9C8
:1018100002BB05BB08BBBD9AC59A909A1C9A1D9A3B
:101820001E9A1F9A04B30F6704BB02B10C6002B981
:10183000AC9AAB9AAA9AA99AA89AAE9AAD9AAC9A7F
:10184000AB9AAA9AA99AA89A1A981B9A01B3006708
:1018500001BB9798949A959A9698AC9AAB9AAA9A43
:10186000A99AA89A0895002391F400E000939000AB
:1018700019B902E00BB908E10AB920FB0EF4579A36
:1018800006E0009395000FEF0CB95E9A08950130C1
:10189000E9F400E0009398001093990002E00093AF
:1018A0009B0008E100939A0020FB2EF400919A001F
:1018B000006800939A0006E000939D000FEF0093EC
:1018C0009C0000919B00006400939B000895592F99
:1018D000482F80E090E008C02FE93FE021503040E1
:1018E000E9F700C00000019680179107A8F3842F44
:1018F000952F08959A938A9380E090E098D20A33C6
:1019000018F00753102F02C00053102F012F10E0C2
:10191000102F00E0110F110F110F110F802B912BC1
:1019200086D20A3318F00753102F02C00053102F2D
:10193000012F302F20E0822B932B79D20A3318F01D
:101940000753102F02C00053102F012F10E044E066
:101950000E94214E802B912B6AD20A3318F0075334
:10196000102F02C00053102F012F10E0802B912B5D
:101970008C018991999108950E94C34E24972A83DE
:101980003B83B02FD12E7A0182E090E001E00093FA
:10199000F30CBB249699B394CC249599C394969A4E
:1019A000959825C0949801E010E091DF00E0009345
:1019B000090D0093080D949A05E010E088DF01E21C
:1019C00005D101E311E083DF08E000D10091080DAB
:1019D0001091090D011751F00091080D1091090D9A
:1019E000011721F024D20132B9F791E08A958130B4
:1019F00010F09923B9F2992309F4B1C000E00093E3
:101A0000090D0093080D4424552466247724A0E092
:101A10008824992409E6DAD008E0D8D008D20A331D
:101A2000E9F705D2088303D2098301D20A33E9F723
:101A300061DF2801FCD10A33E9F75CDF3801088156
:101A4000003319F40981063431F002E6BFD000E317
:101A5000BDD006E6BBD00FEF60160FEF700649F061
:101A6000E6D10A33E9F7E3D1093511F4A1E001C069
:101A7000A0E00EE110E02BDF00E00093090D0093E1
:101A8000080D02E5A3D008E0A1D0D1D1802F8C367B
:101A900041F4CDD10A33E9F72DDF4801AA24A394FC
:101AA00003C08F3691F7AA24EDEEFCE0408251820C
:101AB000EFEEFCE060827182E1EFFCE080829182D7
:101AC000B0FBC6F404E110E002DF04E47FD008E0DC
:101AD0007DD0ADD10A33E9F705E010E0F8DE0A81E8
:101AE0001B817BD108E072D008E070D008E06ED096
:101AF00008E06CD0B1FB4EF404E110E0E8DEDA1649
:101B000021F007E563D008E061D0B2FBCEF4AA2053
:101B1000B9F004E110E0DBDE03E458D008E056D071
:101B200086D10A33E9F705E010E0D1DE870155D10F
:101B300008E04CD008E04AD008E048D008E046D0A1
:101B400004E110E0C4DE05E441D008E03FD0949801
:101B500001E010E0BCDE949A04E610E0B8DE00E09C
:101B60000093090D0093080D0B2D00FD969A00FFC0
:101B700096980C2D00FD959A00FF959800E0009333
:101B8000F30C092F2496E0E10C94D44E5E9A1B9836
:101B90001A9A18D05E9BFECF1A981B9A08958A93C2
:101BA000802F082F02950F70005D0A3308F0095F3F
:101BB0000DD08F70805D082F0A3308F0095F06D0C2
:101BC000899108955D9BFECF0CB90895A998109155
:101BD0009B00212F25FFFBCF00939C0008959A9333
:101BE0008A93802F082F44E60E94034E902F092FDE
:101BF000005DECDF04E6909F8019082F4AE00E9408
:101C0000034E902F092F005DE1DF0AE0909F8019BD
:101C1000805D082FDBDF8991999108950E94C54E60
:101C200048015901DD24BB2052F49094A094B09453
:101C3000000B8194900AA00AB00A0DE2C7DF80E091
:101C40009AECAAE9BBE3CC241AC0DD2019F082018A
:101C5000005DBCDF82019301AC01BD010E94524EC8
:101C6000801A910AA20AB30A8C019D014AE050E051
:101C700060E070E00E949C4EC801D901C39409E065
:101C8000C016A8F484019501AC01BD010E949C4ED0
:101C9000402E552466247724042D0529062907297A
:101CA000A1F28201005D92DFDD24D394D3CF8401C1
:101CB0009501AC01BD010E949C4E402E5524662426
:101CC0007724042D005D82DFEEE00C94D64E0E9456
:101CD000CB4E38015524A0E1B7E244240FC000E305
:101CE00075DF8C01AD010E94114E601A710A8D01E1
:101CF0004AE050E00E942D4ED801439405E0401682
:101D0000D0F48301AD010E942D4EC801082F092B8C
:101D100031F0082F005D5ADF55245394E2CF55204F
:101D200021F0082F005D52DFDCCF04E04016B8F64A
:101D300000E24CDFD6CFE8E00C94DC4E10916A094B
:101D4000112311F02CDF089523E010E00AD008954C
:101D500020916A09222311F040D0089524E001D097
:101D600008950E94C94E3801822E5524A0E1B7E2A1
:101D700044240FC000E32ADF8C01AD010E94114E04
:101D8000601A710A8D014AE050E00E942D4ED80180
:101D9000439405E04016F0F48301AD010E942D4EFE
:101DA000C80104E010E0242D30E0021B130B99243D
:101DB000081519050CF7082F092B31F0082F005DC5
:101DC00005DF55245394D8CF5520A1F2082F005D8C
:101DD000FDDED2CFEAE00C94DA4E9A938A93C801E2
:101DE0008C01012F10E0DBDE082FD9DE899199915B
:101DF00008950E94CF4EC801D9018C019D01022F88
:101E0000132F330F220B330BE8DF8C01E6DFE4E006
:101E10000C94E04EBA93AA93D80103C00C91D6DE7D
:101E200011960C910023D1F7A991B99108950091D1
:101E3000090D1091080D0117D1F30091090D102F14
:101E400013951093090D10E00F701070F801E65F04
:101E5000F24F008108958A93802F082FC0DE08E298
:101E6000B5DE00E3B3DE08E5B1DE082F98DE09E257
:101E7000ADDE899108950E94C84EEF97EF97EF97D6
:101E80002797A898992401E00093730901E0009333
:101E9000720905C004E110E01ADD08E001BD9920D7
:101EA00011F00C94391803EA15E0B4DF00916309CE
:101EB000D2DF0CEA15E0AEDF20E08E0108571F4F9D
:101EC0000E94EA1F00E00883AE0148575F4F9E0161
:101ED000205F3F4F8E010E943E1E802E00917009B0
:101EE000009371098820D9F20FE1801610F00EE1FD
:101EF000802E28E536E08E010E941C1E002351F63C
:101F000026E536E08E010E941C1E002309F450C015
:101F100007EB10E00E945B4C80E01CC0FE01709655
:101F2000082F10E0000F111F000F111FE00FF11F0D
:101F3000008111812281338190E0FC01EA52F74F48
:101F4000008390E0FC01EA52F74F0081F7DE00E2E7
:101F50003DDE839590E0E82DF0E031978E179F07E6
:101F6000ECF21B981A9A80E008C090E0FC01EA525B
:101F7000F74F008127DE5E9A839590E0E82DF0E030
:101F800031978E179F078CF35E9BFECF1A981B9A92
:101F90000FEF0E94004A0093740909EC10E00E94C0
:101FA0005B4C2091740902E218E00E940D4B77CF40
:101FB00021E536E08E010E941C1E002371F42EE400
:101FC00036E08E010E941C1E002339F421EA35E020
:101FD0008E010E941C1E002369F100916309083CD8
:101FE000B1F40CE810E00E945B4C088919892A8939
:101FF0003B8931DF0AE3EADD088919892A893B89AF
:10200000102F009163090E94CC3CA2DE48CF0889C2
:1020100019892A893B890093A0070C891D892E897B
:102020003F890093A10722E012E0009163090E941A
:10203000374B35CF2CE935E08E010E941C1E002362
:10204000A9F014E3009163090E94AA4DC801282F4A
:1020500014E1009163090E94B61D892F90E0282F9A
:1020600015E1009163090E94B61D19CF27E935E0FB
:102070008E010E941C1E002331F114E300916309BC
:102080000E94AA4DD80114E1009163090E94AA4D53
:10209000C80116E1009163090E94AA4D080F191F9B
:1020A000169507950A1B1B0B212F27FF04C00195CE
:1020B000006810E001C010E0202F1AE000916309D1
:1020C0000E94B61DECCE23E935E08E010E941C1E55
:1020D000002341F001E000936A090BED15E10E9435
:1020E0005B4CDDCE2FE835E08E010E941C1E0023E4
:1020F00041F000E000936A0900EF15E10E945B4C9B
:10210000CECE2AE835E08E010E941C1E0023A9F0E5
:1021100014E3009163090E94AA4DC801282F16E11B
:10212000009163090E94B61D892F90E0282F17E1C6
:10213000009163090E94B61DB2CE26E835E08E01FB
:102140000E941C1E002339F42EE735E08E010E9408
:102150001C1E0023F9F080E014C0FE017096082FC9
:1021600010E0000F111F000F111FE00FF11F008181
:1021700011812281338190E0FC01E056F84F008309
:102180008395881550F38A94282D13E80EEF0E944A
:10219000374B85CE28E735E08E010E941C1E0023B8
:1021A00071F425E735E08E010E941C1E002339F4EE
:1021B00023E735E08E010E941C1E0023A1F100914F
:1021C0006309083C81F40C891D892E893F89980197
:1021D000488959896A897B898A01102F009163098E
:1021E0000E94B93B5CCE80E014C0FE017096082FBF
:1021F00010E0000F111F000F111FE00FF11F0081F1
:1022000011812281338190E0FC01E056F84F008378
:102210008395881550F38A94282D13E00091630963
:102220000E94374B3CCE2CE635E08E010E941C1EEE
:10223000002301F180E014C0FE017096082F10E029
:10224000000F111F000F111FE00FF11F00811181FE
:102250002281338190E0FC01E056F84F00838395A2
:10226000881550F38A94282D14E0009163090E9488
:10227000374B15CE25E635E08E010E941C1E00234B
:1022800039F421E635E08E010E941C1E0023F9F08E
:1022900080E014C0FE017096082F10E0000F111F9F
:1022A000000F111FE00FF11F008111812281338186
:1022B00090E0FC01E056F84F00838395881550F3B9
:1022C0008A94282D15E00EEF0E94374BE8CD2AE5C1
:1022D00035E08E010E941C1E002381F00C891D89AF
:1022E0002E893F89202F488959896A897B898A01EB
:1022F000102F009163090E94B61DD1CD24E535E071
:102300008E010E941C1E002321F104EF10E00E94A8
:102310005B4C8DDD093719F0093509F0C0CD01E0BE
:10232000801619F40091630904C0088919892A8963
:102330003B8920E016E00E94374B002309F4AFCD23
:1023400001E00093630921E030E0A9010E94FF4D04
:10235000A6CD2DE435E08E010E941C1E0023A1F0C5
:1023600001E0801639F420E017E0009163090E9433
:10237000374B95CD20E017E0488959896A897B89D8
:10238000042F0E94374B8BCD2AE435E08E010E944A
:102390001C1E002339F428E435E08E010E941C1E27
:1023A0000023D9F102E0801619F003E0801681F5D0
:1023B0000EE10093A007088919892A893B890093B7
:1023C000A107088919892A893B89012F10E0009308
:1023D000A20703E08016A9F40C891D892E893F8984
:1023E0000093A3070C891D892E893F89012F10E0D6
:1023F0000093A40725E013E0009163090E94374B86
:102400004ECD23E013E0009163090E94374B47CD86
:102410000BE011E00E945B4C42CD23E435E08E01DD
:102420000E941C1E002379F001E0801619F400912F
:10243000630904C0088919892A893B8920E011E0D1
:102440000E94374B2CCD20E435E08E010E941C1EEB
:10245000002349F103E00093A007088919892A891C
:102460003B890093A10706E311E00E945B4C0091B9
:10247000A10764DC0CE511E00E945B4CD8DC093557
:1024800019F0093709F00BCD22E013E00EEF0E949E
:10249000374B0091A1070093630921E030E0A901C7
:1024A0000E94FF4DFCCC2AE036E08E010E941C1EEB
:1024B000002339F428E036E08E010E941C1E002320
:1024C000E1F000916309083C11F426D6E8CC00E065
:1024D0000093A0070AE30093A10722E012E0009115
:1024E00063090E94374B002309F4D9CC009163099A
:1024F0000E3F09F4D4CC10D6D2CC21E036E08E01C8
:102500000E941C1E002309F4C8C103E0801651F488
:10251000488859886A887B880C891D892E893F895B
:10252000A02E0DC002E0801631F4488859886A88D0
:102530007B88A42C04C00EE81DE00E945B4C02E0E6
:10254000801621F003E0801609F0A9CC00E000938A
:1025500072090093730909B1023289F421E014E091
:102560000EEF0E94C04D0AE010E0B1D901E009B9B8
:102570000093620920E030E0A9010E94FF4D22E2B1
:1025800014E00EEF0E94C04D0AE010E0A0D902E274
:1025900009B90093620920E030E0A9010E94FF4DD3
:1025A00021E014E00EEF0E94C04D0AE010E08FD948
:1025B00001E009B90093620920E030E0A9010E941E
:1025C000FF4D00E00E94764C05C001E711E00E943B
:1025D0005B4C4394A41408F441C1042D0E94EE1DE9
:1025E0000023B9F309B1013049F001E009B90093C2
:1025F000620920E030E0A9010E94FF4D0FEA1DE0D2
:102600000E945B4C042D9ADB90E0992329F591E020
:1026100080E00EC0082F0E94EE1D002341F020E054
:1026200011E0082F0E94374B002309F490E08395B6
:102630008F3180F384E68E3640F7082F0E94EE1D1E
:10264000002341F020E011E0082F0E94374B0023C7
:1026500009F490E08395EFCF06EB1DE00E945B4C00
:1026600080E00FC0841561F090E0FC01EB58F64F5C
:102670000081002329F025E01DE2082F0E94B61DED
:1026800083958F3178F384E60FC0841561F090E074
:10269000FC01EB56F64F0081002329F025E01DE2F6
:1026A000082F0E94B61D83958E3678F300EC1DE04E
:1026B0000E945B4C2FEF1AEF042D0E94B61D2EEFE7
:1026C0001DE2042D0E94B61D002309F47ECF03E015
:1026D000502E02E209B90093620920E030E0A9011E
:1026E0000E94FF4D04E610E0F2D80DE04FDA00E062
:1026F0000E94701D0CE44ADA00E00E94701D1B98D5
:102700001A9A80E090ECA0E0B0E088246624772458
:1027100012C0FC013A2F3BBF069000E00BBF8F5F59
:102720009F4FAF4FBF4F800C002D4CDA5E9A01E0F7
:10273000600E00E0701E0FEF601607E1700648F3B0
:10274000082D40DA5E9A5E9BFECF1A981B9A00E035
:102750000E94701D06E51ADA00E00E94701D00E07C
:1027600001C00395043638F410E0F801EE5DF74F30
:1027700010811D32B1F70395202F01C00395043657
:1027800038F410E0F801EE5DF74F10811D32B1F71B
:10279000039510E001C01395183090F4602F062FB8
:1027A0000395422F242F239570E0FB01EE5DF74F38
:1027B000308150E0FA01EE5DF74F4081341759F354
:1027C000183031F50BEC1DE00E945B4C01E4DED9C2
:1027D00000E00E94701D07E4D9D900E00E94701D3E
:1027E00004E610E074D801E009B90093620920E022
:1027F00030E0A9010E94FF4D20E017E0042D0E9467
:10280000374B0CE211E063D800E000937209E1CE8F
:1028100005ED1DE00E945B4C5A9409F063CF01E482
:10282000B5D900E00E94701D07E4B0D900E00E9415
:10283000701D04E610E04BD801E009B9009362096D
:1028400020E030E0A9010E94FF4D20E017E0042DB8
:102850000E94374B0CE211E03AD8BBCE21E014E0E5
:102860000EEF0E94C04D0AE010E031D801E009B936
:102870000093620920E030E0A9010E94FF4D0E9410
:10288000244C09B10093620920E030E0A9010E94C4
:10289000FF4D01E00093730902CB2CEF35E08E0170
:1028A0000E941C1E002309F440C0B091720900E090
:1028B000009373090093720980E001E0801611F41F
:1028C000AEEF05C0088919892A893B89A02F0CE839
:1028D00010E00E945B4C90E005C00DE277D90DE559
:1028E00075D993959A1788F40BE570D9092F26DAD4
:1028F0000AE36CD920E011E0092F0E94374B002336
:1029000061F30FE463D98395EACF0CE810E00E94ED
:102910005B4C082FA0DA08E512E00E945B4CB093F4
:10292000720901E000937309BACA28EF35E08E01FD
:102930000E941C1E002309F450C001E0801619F407
:10294000A091630905C0088919892A893B89A02FAC
:1029500001E00093720900E00093730903EA11E0BB
:102960000E945B4C80E007E412E00E945B4C0A2F5F
:10297000E5D90091090D1091080D011791F057DA72
:10298000802F823411F0823609F4AA958E3411F02A
:102990008E3609F4A3950BE612E00E945B4C0A2FD9
:1029A000CDD921E019E10A2F0E94C04D04E610E0C4
:1029B0000E94670C20E019E10A2F0E94C04D04E636
:1029C00010E00E94670C813521F0813711F08B31C6
:1029D00081F601E00093730962CA21EF35E08E01B0
:1029E0000E941C1E002309F48EC000E000937309AE
:1029F0000AE0ECD880E001C083958E3F08F078C0F3
:102A000089B920E011E00EEF0E94374B0DE0DED8CF
:102A100080FB1EF40BE2DAD802C00AE2D7D800919C
:102A20007409002309F45DC0A0E056C0B0E0FD01C8
:102A3000EE5DF74F00810F3F09F04DC00A2F10E007
:102A40000F5F1F4FF801EE5DF74F00810F3F09F058
:102A500042C00A2F10E00D5F1F4FF801EE5DF74FE7
:102A600000810230C1F50A2F10E00E5F1F4FF80100
:102A7000EE5DF74F408150E00A2F10E00D5F1F4FD1
:102A8000F801EE5DF74F208130E0240F351F0A2F4B
:102A900010E00B5F1F4FF801EE5DF74F008110E073
:102AA000020F131F0F3F20E01207A9F40CE712E0FA
:102AB0000E945B4C082F42D90FE812E00E945B4C49
:102AC0000A2F10E00E5F1F4FF801EE5DF74F0081F7
:102AD00035D90AE07BD8A39500917409A01708F4B2
:102AE000A5CF0091090D1091080D011709F484CFAD
:102AF0000091620909B901E0009373090DE066D8FD
:102B000000E264D8CCC92CEE35E08E010E941C1E78
:102B1000002391F104E00093A007088919892A890C
:102B20003B890093A10722E013E00EEF0E94374B90
:102B300005E912E00E945B4C00E814E82EE130E069
:102B4000488959896A897B894F5F5F4F6F4F7F4FF3
:102B50000E94764E63D800EB12E00E945B4C08891D
:102B600019892A893B8909B90093620920E030E07C
:102B7000A9010E94FF4D93C924EE35E08E010E9409
:102B80001C1E002309F445C001E0801631F400E169
:102B9000402E55246624772404C0488859886A88C2
:102BA0007B8800EC11E00E945B4C2EC00091710903
:102BB000109170090117A9F080E090E0A0E0B0E06A
:102BC000AA240091710910E0F801E056F94F008144
:102BD000E1E7F9E0108113951083B0D800E20E947C
:102BE000E60D8F5F9F4FAF4FBF4F84159505A6052C
:102BF000B705E0F2AA2041F40DE00E94E60D0AE0DC
:102C00000E94E60DAA24A39480E090E0A0E0B0E04A
:102C1000ECCF2FED35E08E010E941C1E002309F43D
:102C20004AC0488859886A887B888C899D89AE8982
:102C3000BF8904EB12E00E945B4C042D7FD80FEBA0
:102C400012E00E945B4C8C0183D809EC12E00E94D8
:102C50005B4CA0E006C021E018E10A2F0E94C04DA5
:102C6000A3954A16C0F70AED12E00E945B4C0CC017
:102C70002FEF33E01EE10A2F0E94C84DA3954A169C
:102C8000B8F78C010E94670C0091090D1091080D96
:102C9000011709F004C9A0E007C020E030E01EE100
:102CA0000A2F0E94C84DA3954A16B8F78C010E94BE
:102CB000670CA0E0E4CF2BED35E08E01BDD70023FB
:102CC00009F434C100E00093730900916309009393
:102CD000A00721E015E00EEF0E94374B01E08016BF
:102CE00041F520E130E0A9010E94F34D802E80E003
:102CF00090E0E82DF0E031978E179F070CF042C06E
:102D0000E82FF0E07196AF010E94F34D10E020E053
:102D100030E0FE017096482F50E0440F551F440FDD
:102D2000551FE40FF51F008311832283338383959E
:102D3000DFCF05E1801610F004E1802E20E130E0C5
:102D4000082DA9010E94FF4D80E015C0FE0170967C
:102D5000082F10E0000F111F000F111FE00FF11FCF
:102D60000081118122813381E82FF0E07196AF015B
:102D70000E94FF4D839590E0E82DF0E031978E178B
:102D80009F0724F30CE810E00E945B4C0BE50E94C7
:102D9000E60D80E004C00DE50E94E60D839590E00D
:102DA000E82DF0E031978E179F07DCF4FE01709656
:102DB000082F10E0000F111F000F111FE00FF11F6F
:102DC00000811181228133810E949E0E90E0E82DC6
:102DD000F0E032978E179F07F4F60DE20E94E60DA1
:102DE000DDCF0091090D1091080D011709F099C070
:102DF0000CE810E00E945B4C80E019C0FE01709668
:102E0000082F10E0000F111F000F111FE00FF11F1E
:102E10000081118122813381102F009163090E946A
:102E20009B4D0E949E0E00E20E94E60D839590E06D
:102E3000E82DF0E031978E179F079CF6FE01709603
:102E4000082F10E0000F111F000F111FE00FF11FDE
:102E50000081118122813381083CF9F000916309DE
:102E6000043688F1009163090E3668F502E517E132
:102E7000FE017096282F30E0220F331F220F331FE0
:102E8000E20FF31F408151816281738150E0040F92
:102E9000151FF80104910230B1F4FE017096082F5D
:102EA00010E0000F111F000F111FE00FF11F008134
:102EB000118122813381102F009163090E94CC3C43
:102EC0000E94A80EB0CF0AE117E1FE017096282FEC
:102ED00030E0220F331F220F331FE20FF31F408118
:102EE00051816281738150E0040F151FF801049134
:102EF000023009F083CFFE017096082F10E0000F1A
:102F0000111F000F111FE00FF11F0081118122819D
:102F10003381102F009163090E94AA4D0E94A80ED0
:102F200082CF01E0009373090C944F0F26ED35E03A
:102F30008E0182D6002389F1488859886A887B8867
:102F40008C899D89AE89BF8900E000937309A0E058
:102F50004A1698F021E018E10A2F0E94C04DA3956F
:102F6000F7CF2FEF33E01EE10A2F0E94C84DA39543
:102F70004A16B8F78C010E94670CA0E007C020E059
:102F800030E01EE10A2F0E94C84DA3954A16B8F7FB
:102F90008C010E94670CA0E0EBCF22ED35E08E01A2
:102FA0004BD6002369F0088919892A893B89009347
:102FB000630921E030E0A9010E94FF4D0C944F0FFE
:102FC0002DEC35E08E0138D6002331F42BEC35E0C2
:102FD0008E0132D6002321F00E9471490C944F0FCC
:102FE00025EC35E08E0128D6002331F423EC35E0C2
:102FF0008E0122D6002321F00E94A4490C944F0F89
:103000002EEB35E08E0118D6002319F03CD00C943D
:103010004F0F2AEB35E08E010FD6002381F002E03E
:10302000801640F0088919892A893B890E949241BB
:103030000C944F0F01E00E9492410C944F0F23EB30
:1030400035E08E01F9D5002331F42FEA35E08E0109
:10305000F3D5002321F0992493940C944F0F0CE89E
:1030600010E00E945B4C08EE1DE00E945B4C0C944B
:103070004F0F00E000937309EF96EF96EF962796B7
:10308000EBE00C94D94E03E319E00E945B4C05E59C
:1030900019E00E945B4C0BE719E00E945B4C00EAD0
:1030A00019E00E945B4C09EE19E00E945B4C00E3C2
:1030B0001AE00E945B4C07E61AE00E945B4C0DE8A8
:1030C0001AE00E945B4C08EC1AE00E945B4C06E0A0
:1030D0001BE00E945B4C02E21BE00E945B4C0CE494
:1030E0001BE00E945B4C07E81BE00E945B4C0CEC71
:1030F0001BE00E945B4C05E11CE00E945B4C09E573
:103100001CE00E945B4C06E91CE00E945B4C03EE55
:103110001CE00E945B4C08950E94CF4E0091630911
:10312000083C09F0B9C088E103E01EE00E945B4C56
:10313000082F0E942B0F0AE30E94E60D182F009122
:1031400063090E94CC3C0E94A80E839500E21EE019
:103150000E945B4C082F0E942B0F0AE30E94E60D91
:10316000182F009163090E94CC3C0E94A80E839501
:103170000DE31EE00E945B4C082F0E942B0F0AE318
:103180000E94E60D182F009163090E94CC3C0E941A
:10319000A80E839583950AE51EE00E945B4C082FDC
:1031A0000E942B0F0AE30E94E60D182F009163097D
:1031B0000E94CC3C0E94A80E8395839507E71EE0F1
:1031C0000E945B4C082F0E942B0F0AE30E94E60D21
:1031D000182F009163090E94CC3C0E94A80E839591
:1031E00004E91EE00E945B4C082F0E942B0F0AE3AB
:1031F0000E94E60D182F009163090E94CC3C0E94AA
:10320000A80E839501EB1EE00E945B4C082F0E94E4
:103210002B0F0AE30E94E60D182F009163090E940C
:10322000CC3C0E94A80E83950EEC1EE00E945B4CE5
:10323000082F0E942B0F0AE30E94E60D182F009121
:1032400063090E94CC3C0E94A80E83950BEE1EE001
:103250000E945B4C082F0E942B0F0AE30E94E60D90
:10326000182F009163090E94CC3C0E94A80E839500
:10327000839508E01FE00E945B4C082F0E942B0FF3
:103280000AE30E94E60D182F009163090E94CC3CCE
:103290000E94A80E839521C480E008E013E00E94FC
:1032A0005B4C082F0E942B0F0CEA1DE00E945B4C28
:1032B000A82FB0E01596FD01EE5DF74F00810E944A
:1032C0002B0F839507E313E00E945B4C082F0E94AD
:1032D0002B0F0CEA1DE00E945B4CA82FB0E0159666
:1032E000FD01EE5DF74F00810E942B0F839506E5EF
:1032F00013E00E945B4C082F0E942B0F0CEA1DE08C
:103300000E945B4CA82FB0E01596FD01EE5DF74FD3
:1033100000810E942B0F839505E713E00E945B4C10
:10332000082F0E942B0F0CEA1DE00E945B4CA82F77
:10333000B0E01596FD01EE5DF74F00810E942B0F66
:10334000839504E913E00E945B4C082F0E942B0F29
:103350000CEA1DE00E945B4CA82FB0E01596FD0121
:10336000EE5DF74F00810E942B0F839503EB13E076
:103370000E945B4C082F0E942B0F0CEA1DE00E945C
:103380005B4CA82FB0E01596FD01EE5DF74F008174
:103390000E942B0F839502ED13E00E945B4C082FD7
:1033A0000E942B0F0CEA1DE00E945B4CA82FB0E09E
:1033B0001596FD01EE5DF74F00810E942B0F83955E
:1033C00001EF13E00E945B4C082F0E942B0F0CEAC8
:1033D0001DE00E945B4CA82FB0E01596FD01EE5D4C
:1033E000F74F00810E942B0F839500E114E00E94AB
:1033F0005B4C082F0E942B0F0CEA1DE00E945B4CD7
:10340000A82FB0E01596FD01EE5DF74F00810E94F8
:103410002B0F83950FE214E00E945B4C082F0E9453
:103420002B0F0CEA1DE00E945B4CA82FB0E0159614
:10343000FD01EE5DF74F00810E942B0F83950EE496
:1034400014E00E945B4C082F0E942B0F0CEA1DE039
:103450000E945B4CA82FB0E01596FD01EE5DF74F82
:1034600000810E942B0F83950DE614E00E945B4CB7
:10347000082F0E942B0F0CEA1DE00E945B4CA82F26
:10348000B0E01596FD01EE5DF74F00810E942B0F15
:1034900083950CE814E00E945B4C082F0E942B0FD0
:1034A0000CEA1DE00E945B4CA82FB0E01596FD01D0
:1034B000EE5DF74F00810E942B0F83950BEA14E01D
:1034C0000E945B4C082F0E942B0F0CEA1DE00E940B
:1034D0005B4CA82FB0E01596FD01EE5DF74F008123
:1034E0000E942B0F83950AEC14E00E945B4C082F7E
:1034F0000E942B0F0CEA1DE00E945B4CA82FB0E04D
:103500001596FD01EE5DF74F00810E942B0F83950C
:1035100009EE14E00E945B4C082F0E942B0F0CEA6E
:103520001DE00E945B4CA82FB0E01596FD01EE5DFA
:10353000F74F00810E942B0F839508E015E00E9451
:103540005B4C082F0E942B0F0CEA1DE00E945B4C85
:10355000A82FB0E01596FD01EE5DF74F00810E94A7
:103560002B0F839507E215E00E945B4C082F0E9409
:103570002B0F0CEA1DE00E945B4CA82FB0E01596C3
:10358000FD01EE5DF74F00810E942B0F839506E44D
:1035900015E00E945B4C082F0E942B0F0CEA1DE0E7
:1035A0000E945B4CA82FB0E01596FD01EE5DF74F31
:1035B00000810E942B0F839505E615E00E945B4C6D
:1035C000082F0E942B0F0CEA1DE00E945B4CA82FD5
:1035D000B0E01596FD01EE5DF74F00810E942B0FC4
:1035E000839504E815E00E945B4C082F0E942B0F86
:1035F0000CEA1DE00E945B4CA82FB0E01596FD017F
:10360000EE5DF74F00810E942B0F839503EA15E0D2
:103610000E945B4C082F0E942B0F0CEA1DE00E94B9
:103620005B4CA82FB0E01596FD01EE5DF74F0081D1
:103630000E942B0F839502EC15E00E945B4C082F33
:103640000E942B0F0CEA1DE00E945B4CA82FB0E0FB
:103650001596FD01EE5DF74F00810E942B0F8395BB
:1036600001EE15E00E945B4C082F0E942B0F0CEA24
:103670001DE00E945B4CA82FB0E01596FD01EE5DA9
:10368000F74F00810E942B0F83950EEE12E00E94EF
:103690005B4C0E94170F00E016E00E945B4C082F65
:1036A0000E942B0F0CEA1DE00E945B4CA82FB0E09B
:1036B0001596FD01EE5DF74F00810E942B0F83955B
:1036C0000CE216E00E945B4C082F0E942B0F0CEAC4
:1036D0001DE00E945B4CA82FB0E01596FD01EE5D49
:1036E000F74F00810E942B0F83950BE416E00E9498
:1036F0005B4C082F0E942B0F0CEA1DE00E945B4CD4
:10370000A82FB0E01596FD01EE5DF74F00810E94F5
:103710002B0F83950AE616E00E945B4C082F0E944F
:103720002B0F0CEA1DE00E945B4CA82FB0E0159611
:10373000FD01EE5DF74F00810E942B0F839509E894
:1037400016E00E945B4C082F0E942B0F0CEA1DE034
:103750000E945B4CA82FB0E01596FD01EE5DF74F7F
:1037600000810E942B0F839508EA16E00E945B4CB3
:10377000082F0E942B0F0CEA1DE00E945B4CA82F23
:10378000B0E01596FD01EE5DF74F00810E942B0F12
:10379000839507EC16E00E945B4C082F0E942B0FCC
:1037A0000CEA1DE00E945B4CA82FB0E01596FD01CD
:1037B000EE5DF74F00810E942B0F839506EE16E019
:1037C0000E945B4C082F0E942B0F0CEA1DE00E9408
:1037D0005B4CA82FB0E01596FD01EE5DF74F008120
:1037E0000E942B0F839505E017E00E945B4C082F89
:1037F0000E942B0F0CEA1DE00E945B4CA82FB0E04A
:103800001596FD01EE5DF74F00810E942B0F839509
:1038100004E217E00E945B4C082F0E942B0F0CEA79
:103820001DE00E945B4CA82FB0E01596FD01EE5DF7
:10383000F74F00810E942B0F839503E417E00E944D
:103840005B4C082F0E942B0F0CEA1DE00E945B4C82
:10385000A82FB0E01596FD01EE5DF74F00810E94A4
:103860002B0F839502E617E00E945B4C082F0E9405
:103870002B0F0CEA1DE00E945B4CA82FB0E01596C0
:10388000FD01EE5DF74F00810E942B0F839501E84B
:1038900017E00E945B4C082F0E942B0F0CEA1DE0E2
:1038A0000E945B4CA82FB0E01596FD01EE5DF74F2E
:1038B00000810E942B0F839500EA17E00E945B4C69
:1038C000082F0E942B0F0CEA1DE00E945B4CA82FD2
:1038D000B0E01596FD01EE5DF74F00810E942B0FC1
:1038E00083950FEB17E00E945B4C082F0E942B0F73
:1038F0000CEA1DE00E945B4CA82FB0E01596FD017C
:10390000EE5DF74F00810E942B0F83950EED17E0BF
:103910000E945B4C082F0E942B0F0CEA1DE00E94B6
:103920005B4CA82FB0E01596FD01EE5DF74F0081CE
:103930000E942B0F83950DEF17E00E945B4C082F20
:103940000E942B0F0CEA1DE00E945B4CA82FB0E0F8
:103950001596FD01EE5DF74F00810E942B0F8395B8
:103960000CE118E00E945B4C082F0E942B0F0CEA20
:103970001DE00E945B4CA82FB0E01596FD01EE5DA6
:10398000F74F00810E942B0F83950BE318E00E94F4
:103990005B4C082F0E942B0F0CEA1DE00E945B4C31
:1039A000A82FB0E01596FD01EE5DF74F00810E9453
:1039B0002B0F83950AE518E00E945B4C082F0E94AC
:1039C0002B0F0CEA1DE00E945B4CA82FB0E015966F
:1039D000FD01EE5DF74F00810E942B0F839509E7F3
:1039E00018E00E945B4C082F0E942B0F0CEA1DE090
:1039F0000E945B4CA82FB0E01596FD01EE5DF74FDD
:103A000000810E942B0F839508E918E00E945B4C0F
:103A1000082F0E942B0F0CEA1DE00E945B4CA82F80
:103A2000B0E01596FD01EE5DF74F00810E942B0F6F
:103A3000839507EB18E00E945B4C082F0E942B0F28
:103A40000CEA1DE00E945B4CA82FB0E01596FD012A
:103A5000EE5DF74F00810E942B0F839506ED18E075
:103A60000E945B4C082F0E942B0F0CEA1DE00E9465
:103A70005B4CA82FB0E01596FD01EE5DF74F00817D
:103A80000E942B0F839505EF18E00E945B4C082FD6
:103A90000E942B0F0CEA1DE00E945B4CA82FB0E0A7
:103AA0001596FD01EE5DF74F00810E942B0F839567
:103AB00004E119E00E945B4C082F0E942B0F0CEAD6
:103AC0001DE00E945B4CA82FB0E01596FD01EE5D55
:103AD000F74F00810E942B0F8395E4E00C94E04E99
:103AE0009A938A93902F80E0009171091091700948
:103AF0000117D1F340E050E060E070E000917109FF
:103B0000109170090117A1F48A019B01A801B90164
:103B10004F5F5F4F6F4F7F4F013EE3E91E07E4E0C9
:103B20002E07E0E03E0750F3082F89919991089500
:103B30000091710910E0F801E056F94F0081E1E7CA
:103B4000F9E0108113951083282F30E0F901EE5D24
:103B5000F74F0083992341F0082F10E0F801EE5D44
:103B6000F74F00810E94E60D8395C4CF0E94CF4E8F
:103B7000902FA12FB22FA093A007B093A10700EF21
:103B80000093A20705E50093A3070FE00093A407A5
:103B90000AEA0093A50726E01DE0092F0E94BC4A0F
:103BA000802F00917309002349F00CE810E00E9477
:103BB0005B4C282F06ED18E00E940D4B05E010E04D
:103BC0000E94670C1A2F092F0E949B4D0B1711F4AE
:103BD00001E001C000E0E4E00C94E04E0F3130F46D
:103BE00010E0F801EB58F64F00810895043650F0CC
:103BF0000E3640F410E004561040F801EB56F64F34
:103C00000081089500E00895A80100E001C0039537
:103C1000083C88F410E0F901E00FF11F608110E02A
:103C2000FA01E00FF11F608310E0F901E00FF11FCE
:103C30001081112361F70895A80100E010E0FA0156
:103C4000E00FF11F608110E0F901E00FF11F10811A
:103C5000611791F4039510E0FA01E00FF11F108154
:103C6000112339F410E0F901E00FF11F1081112345
:103C700021F0093C18F3089500E008950E94CC4E0D
:103C8000D901CA01442401C043945524FC01E40D28
:103C9000F51D20812032C1F32CE3421608F041C00B
:103CA0005524FC01E40DF51D20812223D1F120E0F3
:103CB00021C05524FC01E40DF51D3081313670F032
:103CC0005524FC01E40DF51D30813B3738F45524B3
:103CD000FC01E40DF51D30813F7530835524FC0156
:103CE000E40DF51D408130E0F801E20FF31F408341
:103CF000239543945524FC01E40DF51D30813033A8
:103D000050F05524FC01E40DF51D30813B3718F4CB
:103D100030E1431670F240E030E0F801E20FF31FAB
:103D20004083E02FF12F0081002311F400E0A6C0B2
:103D300066249EC043945524FC01E40DF51D0081CA
:103D40000032C1F35524FC01E40DF51D0081002370
:103D500019F46394062D92C000E010E020E030E0FA
:103D6000462D50E0440F551F440F551FFD01E40F31
:103D7000F51F008311832283338342C0062D10E098
:103D8000000F111F000F111FFD01E00FF11F008137
:103D90001181228133814AE050E060E070E00E94AE
:103DA000524E462D50E0440F551F440F551FFD0144
:103DB000E40FF51F00831183228333835524FC0114
:103DC000E40DF51D008110E000531040212F220F5B
:103DD000220B322F462D50E0440F551F440F551F24
:103DE000FD01E40FF51F4081518162817381400F15
:103DF000511F621F731F40835183628373834394F7
:103E00000CE34016A0F55524FC01E40DF51D0081DE
:103E1000002321F402E0600E062D30C05524FC0181
:103E2000E40DF51D00810B33E1F05524FC01E40D98
:103E3000F51D00810A33A9F05524FC01E40DF51DA0
:103E400000810C3271F05524FC01E40DF51D008158
:103E50000E3239F05524FC01E40DF51D00810032CD
:103E600081F400E25524FC01E40DF51D0083639408
:103E70000EE1601608F45FCF6394062DE7E00C9422
:103E8000DD4E00916A09002309F478CF5524FC0126
:103E9000E40DF51D0081003308F446C05524FC01F3
:103EA000E40DF51D00810A33F8F5062D10E0000F32
:103EB000111F000F111FFD01E00FF11F0081118183
:103EC0002281338144E00E946E4E462D50E0440F23
:103ED000551F440F551FFD01E40FF51F008311838B
:103EE000228333835524FC01E40DF51D008110E08D
:103EF00000531040212F220F220B322F462D50E06D
:103F0000440F551F440F551FFD01E40FF51F40815D
:103F1000518162817381400F511F621F731F408363
:103F20005183628373836BCF5524FC01E40DF51D2F
:103F30000081013408F463CF5524FC01E40DF51D24
:103F400000810B3708F05BCF5524FC01E40DF51D13
:103F500000810F750083062D10E0000F111F000F68
:103F6000111FFD01E00FF11F0081118122813381BA
:103F700044E00E946E4E462D50E0440F551F440F02
:103F8000551FFD01E40FF51F008311832283338346
:103F90005524FC01E40DF51D008110E0075310408D
:103FA000212F220F220B322F462D50E0440F551F98
:103FB000440F551FFD01E40FF51F408151816281BF
:103FC0007381400F511F621F731F408351836283AF
:103FD000738315CF0E94CF4EC801A22FB1E016C047
:103FE00008E00E94E60D00E20E94E60D08E00E9453
:103FF000E60D0A2FA02FAA95002391F729EE3DE0A8
:104000008C0102DEA02F8C010E940A0FBB23A9F1B4
:104010000E94170F102F1050C9F31A9551F3175023
:1040200099F0125029F0135019F01E5079F319C06D
:1040300000E0B0E0FC01EA0FFB1F00839C0109EEE9
:104040001DE0E2DD01E01AC0A13000F3AA9508E00E
:104050000E94E60D00E20E94E60D08E00E94E60DD7
:10406000D5CFAC3398F62A2F30E0FC01E20FF31FD6
:1040700000830E94E60DA395C9CF00E0E4E00C9414
:10408000E04E0E94CF4E902F812F983050F588300F
:1040900040F5092F10E00F5F1F4F40E450E00E94F1
:1040A000114ED801082F10E00F5F1F4F40E450E081
:1040B0000E94114E20E011C0422F50E0400F511FCE
:1040C000FA01E052F64F3081422F50E04A0F5B1F59
:1040D000FA01E052F64F30832395203468F3092F1C
:1040E00003D0E4E00C94E04E9A938A93902F97309B
:1040F00011F490E001C0939580E007C0182F092FBC
:1041000050D2182F092F2BD183958F31B8F31FE18F
:10411000092F47D21FE1092FD3D0F801E052F64F03
:1041200000810E949E0E10E2092F3BD210E2092F5F
:10413000C7D0F801E052F64F00810E949E0E89918F
:1041400099910895005049F00A9561F00A9579F027
:104150000A9591F00A95A9F008950BED14E10E94DB
:104160005B4C08950FEE14E10E945B4C08950DEF37
:1041700014E10E945B4C089500E115E10E945B4C44
:10418000089500E215E10E945B4C08959A938A938A
:10419000802F912FE7E1F6E11491EEE0F6E1049132
:1041A0000E94E72F22E0082F10E00E94B10EE8E104
:1041B000F6E11491EFE0F6E104910E94E72F22E08E
:1041C000092F10E00E94B10EE9E1F6E11491E0E15F
:1041D000F6E104910E94E72F192F082F71D00E9459
:1041E000A80E8991999108958A93E1E1F6E11491DD
:1041F000E8E0F6E104910E94E72F80E004C000E2CD
:104200000E94E60D83958634D0F3E1E1F6E1149146
:10421000E8E0F6E104910E94E72F899108959A93CE
:104220008A939091F40980E00CC0182F0091250E1C
:104230000395B7D108E00E94E60D00E20E94E60D6A
:1042400083958F3190F380E00BC0182F092F0395D1
:10425000A8D108E00E94E60D0CE70E94E60D8395C8
:104260008F3198F39093250EE5E1F6E11491ECE09F
:10427000F6E104910E94E72F092F0E949E0E89917A
:1042800099910895093031F4133020F0143110F46D
:1042900001E00895083021F41F3110F401E0089581
:1042A000083030F4103211F01F3111F401E008959C
:1042B000083020F4103210F402E0089500E0089570
:1042C000682F202F812F222371F48F3138F4082F8B
:1042D00010E0000F111F00501E4F39C0082F10E0D2
:1042E000015E1D4F34C08F3149F4022F10E040E4CD
:1042F00050E00E94114E025C1F4F29C0803249F4E9
:10430000022F10E040E450E00E94114E015C1F4F6C
:104310001EC0283029F4082F10E0005E1F4F17C080
:10432000293029F4082F10E0055F1F4F10C0022F1D
:1043300010E00150104040E450E00E94114E9801FE
:1043400002E0809F8001020F131F005C1F4F0034AA
:1043500022E0120710F000E010E0862F08959A93F3
:104360008A93902F812F8F3108F042C0182F092F88
:10437000A7DFF801E052F64F20813181203004E0C0
:10438000300748F0182F092F9BDFF801E052F64F55
:10439000018107FF0BC0182F092F92DFF801E052AF
:1043A000F64F008111810E94A80E22C0182F092FFC
:1043B00087DFF801E052F64F018105FF0DC00FE3E2
:1043C0000E94E60D0FE30E94E60D0FE30E94E60D4A
:1043D0000FE30E94E60D0CC00DE20E94E60D0DE217
:1043E0000E94E60D0DE20E94E60D0DE20E94E60D30
:1043F0008991999108959A938A930091E50C0023ED
:1044000051F000E09FDE0E94170F093521F00937B7
:1044100011F000E085C0E3EEFCE00081118120E0B6
:1044200030E040E052E060E070E00E94524EA801AF
:10443000B901405050426F4F7F4F90E000E010E0D4
:1044400018C0080122243324040E151E261E371E10
:10445000F001322D3BBF069020E02BBFF801E05267
:10446000F64F0082F801E052F64F2081920F0F5F65
:104470001F4F003022E0120720F380E00DC020E043
:1044800030E402E0809F800100501E4FF801E052AE
:10449000F64F2083318383958F3180F5082F10E00C
:1044A000F801EB58F64F0081002349F318E1082F7B
:1044B0000E949B4D013081F41EE1082F0E94BB2F0A
:1044C00022E0829F20E0020E22E0121EF001E05264
:1044D000F64F00831183DFCF14E2082F0E94BB2F19
:1044E0000060106222E0829F20E0020E22E0121E95
:1044F000F001E052F64F00831183CDCF9F3F21F4AE
:104500000091F409083008F00ED000E00093E50CAB
:104510000091F709053018F000E00093F70901E079
:104520008991999108953B2F2A2FE0E0F0E006C091
:1045300000E0DF01A052B64F0C933196E03200E06C
:10454000F007B0F3E0E2F0E006C005E5DF01A052BD
:10455000B64F0C933196E03400E0F007B0F3E0E49E
:10456000F0E009C000E010E4DF01A052B64F0D9367
:104570001C9311973296E03002E0F00798F300E0C8
:104580000093F40901E00093EF0900E20093F609BB
:1045900000E20093F80900E00093ED09A22FB32F89
:1045A00008959A938A936297602F212FCE010896DF
:1045B000E6E4FEE930E08C014AE050E00E94B24EB1
:1045C000CE01E0E5FEE930E08C0148E050E00E94D9
:1045D000B24E203211F02F3151F42395122FFE01EB
:1045E00070E0E60FF71F00810E94E72F10C02F3107
:1045F00058F42395122FFE01389670E0E60FF71F4E
:1046000000810E94E72F03C001E20E94E60D62963E
:104610008991999108958A93802F03C000E20E94A6
:10462000E60D082F802F8A950023C1F78991089500
:104630000E94D04E80E005C00CE810E00E945B4C68
:1046400083958C33C8F311E001E00E94E72F05E267
:104650001FE00E945B4C0FE31FE00E945B4C07E2EF
:10466000DADF0AE51FE00E945B4C07E61FE00E94CC
:104670005B4C07E2D0DF02E81FE00E945B4C09E8D8
:104680001FE00E945B4C07E2C6DF04EA1FE00E94C5
:104690005B4C02EB1FE00E945B4C07E2BCDF0DECC1
:1046A0001FE00E945B4C0BED1FE00E945B4C07E299
:1046B000B2DF06EF1FE00E945B4C04E010E10E94B5
:1046C0005B4C07E2A8DF0FE110E10E945B4C0DE2BA
:1046D00010E10E945B4C07E29EDF08E410E10E94BB
:1046E0005B4C06E510E10E945B4C07E294DF01E7BA
:1046F00010E10E945B4C0FE710E10E945B4C07E267
:104700008ADF0AE910E10E945B4C08EA10E10E948E
:104710005B4C07E280DF03EC10E10E945B4C01ED93
:1047200010E10E945B4C07E276DF0CEE10E10E9484
:104730005B4C0AEF10E10E945B4C07E26CDF05E185
:1047400011E10E945B4C03E211E10E945B4C07E225
:1047500062DF0EE311E10E945B4C0CE411E10E9468
:104760005B4C07E258DF07E611E10E945B4C05E76E
:1047700011E10E945B4C07E24EDF00E911E10E946B
:104780005B4C0EE911E10E945B4C07E244DF09EB50
:1047900011E10E945B4C07EC11E10E945B4C07E2C7
:1047A0003ADF02EE11E10E945B4C00EF11E10E9442
:1047B0005B4C07E230DF0BE012E10E945B4C09E149
:1047C00012E10E945B4C07E226DF04E312E10E9443
:1047D0005B4C02E412E10E945B4C0DE512E10E9489
:1047E0005B4C08E712E10E945B4C03E912E10E9476
:1047F0005B4C0EEA12E10E945B4C09EC12E10E9454
:104800005B4C04EE12E10E945B4C0FEF12E10E9440
:104810005B4C0AE113E10E945B4C05E313E10E944B
:104820005B4C00E513E10E945B4C0BE613E10E9438
:104830005B4C0091F0090A3029F40CE913E10E9465
:104840005B4C04C006E813E10E945B4C02EB13E1F1
:104850000E945B4CE3EEFCE000811181012B29F406
:104860000DE314E10E945B4C04C00EEE13E10E94C4
:104870005B4C0CE814E10E945B4C80E001C0839526
:104880008132F8F490E006C0A23019F4182F092FF5
:1048900066DD9395933198F7182F092FF3DCA02F3D
:1048A000AA23B9F3182F092F7CDEA13069F7182F3E
:1048B000092F06DDF801E052F64F00810E949E0E9E
:1048C000E8CFADDCE2E1F6E11491E9E0F6E1049134
:1048D0000E94E72F00EE19E00E940A0FE3E1F6E1E3
:1048E0001491EAE0F6E104910E94E72FE3EEFCE088
:1048F000008111810E94A80EE4E1F6E11491EBE041
:10490000F6E104910E94E72FE3EEFCE000811181C3
:1049100020E030E040E052E060E070E00E94524E63
:10492000005010422F4F3F4F0E94F90EE3E00C94CD
:10493000E14E0E94C64EEF97EA97DA95BE016452A7
:104940007F4FE8E5FEE930E08B0141E250E00E9454
:10495000B24EA0E0BA2FBA2ECA2E24EF3FE0A90132
:104960000E94F34D053511F40C94042F1A2F0B2FD0
:104970000DDC1A2F0B2F15DE9090F40900916A09B7
:10498000002319F000E1A02E02C00AE0A02E0E9430
:10499000170F902F9B31D9F50E94170F902F9B3541
:1049A00019F40E94170F902F943421F4BB2389F03F
:1049B000BA950FC0933411F4B3950BC0913421F420
:1049C000AA2339F0AA9505C0923419F4A03208F44C
:1049D000A395FE01E452FF4F0A2F10E0E00FF11FF4
:1049E00000810B1738F4FE01E452FF4FB0E0EA0FEC
:1049F000FB1FB081BC1521F4AB1511F40C949E2F54
:104A00001A2F0B2FC3DBCB2EBA2E0C949E2F903275
:104A100009F044C01A2F0B2F35DC023011F00C9432
:104A20009E2F80E090E21A2F0B2F4ADCF801E05213
:104A3000F64F008111810827192700831183BB23BA
:104A400029F58A2F02E0809F800100501E4FF80157
:104A5000E052F64F018105FD16C090E0FC01EB58D5
:104A6000F64F0081002379F014E2082F0E94BB2F3B
:104A700022E0829F20E0020E22E0121EF001E052AE
:104A8000F64F008311830A2F0E946D3A1A2F0B2FC5
:104A900066DC01E00093E50C0C949E2F9D3509F037
:104AA0004CC01A2F0B2F7DDD1A2F0B2FEBDB0130A3
:104AB000B9F41A2F0B2F04DCF801E052F64F0081F5
:104AC000039500831A2F0B2FFBDBF801E052F64F02
:104AD00000810E949E0E01E00093E50C0C949E2F35
:104AE000023011F00C949E2F1A2F0B2FE9DBF801E6
:104AF000E052F64F008111810F7F13700F3F23E0CA
:104B0000120711F40C949E2F1A2F0B2FD9DBF801EA
:104B1000E052F64F008111810F5F1F4F0083118318
:104B20001A2F0B2F1CDCBB2319F40A2F0E946D3A9D
:104B300001E00093E50C0C949E2F9B3509F04AC0D0
:104B40001A2F0B2F2EDD1A2F0B2F9CDB0130B9F4FF
:104B50001A2F0B2FB5DBF801E052F64F00810A95B2
:104B600000831A2F0B2FACDBF801E052F64F0081C7
:104B70000E949E0E01E00093E50C0C949E2F0230E3
:104B800011F00C949E2F1A2F0B2F9ADBF801E05294
:104B9000F64F008111810F7F1370012B11F40C94DB
:104BA0009E2F1A2F0B2F8CDBF801E052F64F00815D
:104BB000118101501040008311831A2F0B2FCFDB7E
:104BC000BB2319F40A2F0E946D3A01E00093E50C13
:104BD0000C949E2F9D3709F050C01A2F0B2F52DBDB
:104BE0000130B9F41A2F0B2F6BDBF801E052F64FAE
:104BF00000810A0D00831A2F0B2F62DBF801E052AF
:104C0000F64F00810E949E0E01E00093E50C0C948B
:104C10009E2F023011F00C949E2F1A2F0B2F50DB79
:104C2000F801E052F64F008111810F7F13702FEFD2
:104C300033E04A2D50E0241B350B0217130710F008
:104C40000C949E2F8A2D90E01A2F0B2F39DBF80140
:104C5000E052F64F00811181080F191F0083118364
:104C60001A2F0B2F7CDBBB2319F40A2F0E946D3AFD
:104C700001E00093E50C0C949E2F9B3709F04CC08B
:104C80001A2F0B2FFFDA0130B9F41A2F0B2F18DB74
:104C9000F801E052F64F00810A1900831A2F0B2FFA
:104CA0000FDBF801E052F64F00810E949E0E01E0FA
:104CB0000093E50C0C949E2F023011F00C949E2F63
:104CC0001A2F0B2FFDDAF801E052F64F0081118107
:104CD0000F7F13702A2D30E00217130710F40C9485
:104CE0009E2F8A2D90E01A2F0B2FEADAF801E0525E
:104CF000F64F00811181081B190B008311831A2FB5
:104D00000B2F2DDBBB2319F40A2F0E946D3A01E013
:104D10000093E50C0C949E2F67DA903360F09B377C
:104D200050F4092F0E94E60D98A721E08E01085D3E
:104D30001F4F50D905C020E08E01085D1F4F4AD992
:104D400000E00883AE01485D5F4F9E012C593F4F44
:104D50008E010E943E1E902F992311F40C949E2FD9
:104D600023E935E08E010E941C1E002351F001E072
:104D700000936A09A0E0BA2F1A2F0B2F07DA0C94C0
:104D80009E2F29E436E08E010E941C1E002359F05C
:104D90000AE00093F0094CDCA0E0BA2F1A2F0B2F89
:104DA000F5D90C949E2F23E436E08E010E941C1E40
:104DB000002359F000E00093F0093ADCA0E0BA2F9C
:104DC0001A2F0B2FE3D90C949E2F2FE835E08E017C
:104DD0000E941C1E002351F000E000936A09A0E02D
:104DE000BA2F1A2F0B2FD2D90C949E2F20E436E025
:104DF0008E010E941C1E002341F01ADCA0E0BA2F95
:104E00001A2F0B2FC3D90C949E2F2CE336E08E0162
:104E10000E941C1E002339F424EE35E08E010E940E
:104E20001C1E002391F0E1E1F6E11491E8E0F6E1C7
:104E300004910E94E72F0E943B0FFADBA0E0BA2FFB
:104E40001A2F0B2FA3D90C949E2F27E336E08E0147
:104E50000E941C1E0023B1F0933021F002E072D9B1
:104E60000C949E2FFE01FF9605A116A127A130A547
:104E7000B02FFE01FF9601A512A523A534A5A02FF2
:104E80000C949E2F22E336E08E010E941C1E00230C
:104E900039F420E336E08E010E941C1E002349F104
:104EA000E3EEFCE0208131812F3700E03007E8F4A9
:104EB000E3EEFCE0008111810F5F1F4F008311833F
:104EC0009ADA002341F0B4DBA0E0BA2F1A2F0B2F9F
:104ED0005DD90C949E2FE3EEFCE00081118101501E
:104EE0001040008311830C949E2F01E02BD90C9469
:104EF0009E2F29E236E08E010E941C1E002339F409
:104F000027E236E08E010E941C1E002321F1E3EE11
:104F1000FCE000811181012BD9F0E3EEFCE000817F
:104F20001181015010400083118365DA002339F0AC
:104F30007FDBA0E0BA2F1A2F0B2F28D9FFC7E3EE93
:104F4000FCE0008111810F5F1F4F00831183F6C7C2
:104F500001E0F8D8F3C722E236E08E010E941C1E61
:104F6000002339F420E236E08E010E941C1E00234B
:104F700099F1923019F002E0E5D8E0C7FE01FF9602
:104F800005A116A127A130A5003840E0140740E094
:104F9000240740E03407E8F4E3EEFCE080819181EF
:104FA000FE01FF9605A116A127A130A5E3EEFCE0C6
:104FB0000083118320DA002339F03ADBA0E0BA2F16
:104FC0001A2F0B2FE3D8BAC7E3EEFCE0808391835E
:104FD000B5C701E0B7D8B2C72BE136E08E010E9419
:104FE0001C1E0023D1F1923019F002E0ABD8A6C705
:104FF000FE01FF9605A116A127A130A5003840E0CB
:10500000140740E0240740E0340720F5E3EEFCE01D
:1050100080819181FE01FF9605A116A127A130A5EF
:10502000E3EEFCE000831183E6D9002371F0E3EEA8
:10503000FCE080839183FCDAA0E0BA2F1A2F0B2FBB
:10504000A5D801E00093E50C79C7E3EEFCE080838E
:10505000918374C701E076D871C728E536E08E01E8
:105060000E941C1E0023E1F00091E50C002389F052
:1050700000E068D80E94170F902F993519F09937E2
:1050800009F05CC704E110E00E94670C08E001BD74
:1050900055C704E110E00E94670C08E001BD4EC74F
:1050A00026E136E08E010E941C1E002319F10AE35E
:1050B0000E94E60D20E08E01085D1F4F0E94EA1F4E
:1050C000002361F000E00DAB9E01285D3F4F00EE34
:1050D00019E00E94041E01E00093E50CE2E1F6E114
:1050E0001491E9E0F6E1049172D700EE19E00E9414
:1050F0000A0F24C723E136E08E010E941C1E002304
:1051000009F482C09130A9F580E08F3108F016C70C
:1051100002E0809F00E0000E02E0101EF001E0526D
:10512000F64F018105FF23C090E0FC01EB58F64FDC
:1051300000810023E1F021E018E1082F0E94C04D1A
:1051400014E2082F18D722E0829F20E0020E22E00E
:10515000121EF001E052F64F00831183082F0E94C7
:105160006D3A182F00E01DDA182F00E0F8D883956B
:10517000CCCF44245524E92FF0E031974E165F063A
:105180000CF0DCC6FE01EC59FF4F042D10E0000FBF
:10519000111F000F111FE00FF11F008111812281EB
:1051A0003381802F02E0809F00E0000E02E0101E9D
:1051B000F001E052F64F018105FF24C0082F10E0F6
:1051C000F801EB58F64F00810023E1F021E018E1EF
:1051D000082F0E94C04D14E2082FCDD622E0829FF6
:1051E00020E0020E22E0121EF001E052F64F008392
:1051F0001183082F0E946D3A182F00E0D2D9182F82
:1052000000E0ADD84394B6CF2FE036E08E010E9487
:105210001C1E002309F460C0913021F580E08F311D
:1052200008F08CC690E0FC01EB58F64F008100239B
:10523000B9F020E018E1082F0E94C04D02E0809FE5
:1052400000E0000E02E0101EF001E052F64F018176
:1052500000620183182F00E0A4D9182F00E07FD846
:105260008395DDCF44245524E92FF0E031974E1685
:105270005F060CF063C6FE01EC59FF4F042D10E0F1
:10528000000F111F000F111FE00FF11F008111818E
:1052900022813381802F082F10E0F801EB58F64F60
:1052A00000810023B9F020E018E1082F0E94C04DD2
:1052B00002E0809F00E0000E02E0101EF001E052CC
:1052C000F64F018100620183182F00E06AD9182F80
:1052D00000E045D84394C7CF28E936E08E010E940C
:1052E0001C1E002309F466C0913009F048C00091EB
:1052F000090D1091080D011709F020C608EC10E007
:105300000E94670C0E94F420E1E1F6E11491E8E0CC
:10531000F6E104915CD612E206E60E949B4D0E94E3
:105320009E0E00E20E94E60D13E206E60E949B4DEF
:105330000E949E0E00E20E94E60D14E206E60E9424
:105340009B4D0E949E0E0CE20E94E60D12E205E6C5
:105350000E949B4D0E949E0E00E20E94E60D13E209
:1053600005E60E949B4D0E949E0E00E20E94E60D03
:1053700014E205E60E949B4D0E949E0EB8CF92302B
:1053800009F0DCC580E007C000E090E0FC01E954D2
:10539000F24F008383958F31B8F3FE01FF9605A18C
:1053A00016A127A130A50093E20C0EE215E10E94A0
:1053B0005B4CC4C523E936E08E010E941C1E00230D
:1053C00039F421E936E08E010E941C1E0023C1F051
:1053D000FE01FF9605A116A127A130A5923021F06C
:1053E00002E00E94A220AAC5083020F004E00E943A
:1053F000A220A4C50093F40901E00093E50C9EC52A
:105400002CE836E08E010E941C1E002399F1933097
:1054100021F002E00E94A22091C5FE01FF9605A1A5
:1054200016A127A130A5802FFE01FF9601A512A588
:1054300023A534A5902F983010F4883020F004E094
:105440000E94A2207BC50AE30E94E60D082F0E945D
:105450009E0E0DE20E94E60D0EE30E94E60D092F5E
:105460000E949E0E182F092F0E94412001E00093F8
:10547000E50C64C528E735E08E010E941C1E002360
:1054800041F423E735E08E010E941C1E002309F43D
:1054900088C0933020F002E00E94A2204FC59130D6
:1054A00019F40091F40906C0FE01FF9605A116A1AA
:1054B00027A130A5073020F004E00E94A2203EC5BD
:1054C000E3EEFCE020813181232B41F41091F409BB
:1054D000133020F004E00E94A22030C5923039F44D
:1054E00017E00E94412001E00093E50C19C09130C3
:1054F000A1F40091F409073080F417E00091F40959
:105500000E944120E0EEF9E004890395048B0E949B
:105510000F2101E00093E50C03C004E00E94A220EB
:10552000E3EEFCE000811181012B09F007C5009139
:10553000F409013029F00091F409023009F0FEC4A9
:1055400000E410E020E830E040EC50E080E01EC0D5
:1055500062E0869F020E131EF001E052F64F20809B
:10556000318062E0869F000E111EF001E052F64F7E
:1055700060817181261A370A62E0869F040E151E2B
:10558000F001E052F64F2082318283958F3100F393
:105590000E94F42003E00E94A22002E00E947420F6
:1055A000CDC425E836E08E010E941C1E002339F48C
:1055B00028E036E08E010E941C1E0023E9F19230A3
:1055C00029F5FE01FF9605A116A127A130A5802F80
:1055D000873020F004E00E94A220B0C40091F409BA
:1055E000801770F4E0EEF9E004890A95048B0E94BC
:1055F0000F2106C0182F1395082F0E944120839574
:105600008630C0F301E00093E50C98C4913009F0B6
:1056100095C40091F409013058F0E0EEF9E00489F6
:105620000A95048B0E940F2101E00093E50C86C4CB
:1056300004E00E94A22082C42EE736E08E010E9480
:105640001C1E002339F42CE736E08E010E941C1E3C
:10565000002389F1FE01FF9605A116A127A130A51F
:10566000802F923021F002E00E94A22067C4873090
:1056700020F004E00E94A22061C406E0402E06C093
:10568000142D1A95042D0E9441204A948415C0F3CC
:1056900017E0082F0E9441200091F409801738F488
:1056A000E0EEF9E004890395048B0E940F2101E0EC
:1056B0000093E50C43C42AEB35E08E010E941C1ECA
:1056C000002379F0923048F0FE01FF9605A116A163
:1056D00027A130A50E94924131C401E00E9492416D
:1056E0002DC42AE435E08E010E941C1E002341F4E3
:1056F00028E435E08E010E941C1E002309F461C0DD
:10570000FE01FF9605A116A127A130A5402E9230DB
:1057100021F002E00E94A22011C407E0401620F010
:1057200004E00E94A2200AC499E580E01DC0082F71
:1057300010E0F801EB58F64F00810023A1F0042D92
:1057400010E040E450E00E94114E22E0829F000EE3
:10575000111E00E4000E00E0101EF001E052F64FB2
:10576000018106FD9EE483958F3108F30091F409D1
:10577000401640F0993531F400E00E94A2200E94CA
:10578000170F902F993519F0993709F0D7C3E6E133
:10579000F6E11491EDE0F6E1049119D4042D0E9494
:1057A0009E0E07E00E947420142D07E00E94412005
:1057B00080E08F3108F0C2C3082F0E946D3A8395B4
:1057C000F8CF27E736E08E010E941C1E002309F463
:1057D000BAC0E3EEFCE040805180913061F4E3EE2A
:1057E000FCE00081118120E030E0FE01FF9605A37E
:1057F00016A327A330A7EFEDFDE0208131812733E9
:1058000002E0300738F023E333E012E20EEF0E94AB
:10581000C84D06C02FEF33E012E20EEF0E94C84DD4
:1058200000E010E0E3EEFCE00083118380E00CC0B8
:1058300022E0829F20E0020E22E0121EF001E052E0
:10584000F64F0083118383958F3100F590E0FC01C2
:10585000EB58F64F00810023B1F318E1082F0E94A6
:105860009B4D013021F41EE1082F85D303C014E2C3
:10587000082F81D3003020E41207D1F60DED1DE092
:105880000E945B4C082F0E949E0EDDCFE3EEFCE0F1
:1058900040825182FE01FF9605A116A127A130A5E5
:1058A000A6D407C001E00093E60C05EF1DE00E94BE
:1058B0005B4C0091E80C0023A1F00091090D1091C0
:1058C000080D0117B1F30E94170F0B3159F30D307A
:1058D00081F702E00093E60C0CEF1DE00E945B4CA8
:1058E000E8CF0EE215E10E945B4C04EF11E00E944C
:1058F000670C80E00CC022E0829F20E0020E22E0D4
:10590000121EF001E052F64F0083118383958F3110
:10591000B0F490E0FC01EB58F64F00810023B1F3A6
:105920001EE1082F28D3003020E4120721F70DEDE7
:105930001DE00E945B4C082F0E949E0EE7CF07E0FF
:105940000E947420FBC223E736E08E010E941C1ED9
:10595000002309F457C0923051F4FE01FF9605A1CF
:1059600016A127A130A5003024E0120720F002E0A4
:105970000E94A220E3C21A2F0B2F0E94D1221A2FBD
:105980000B2F0E9442210130E9F4FE01FF9605A190
:1059900016A127A130A5802F1A2F0B2F0E9460215E
:1059A000F801E052F64F80831A2F0B2F0E946021DE
:1059B000F801E052F64F00810E949E0E01E0009334
:1059C000E50CBCC2023009F0B9C2FE01FF9605A188
:1059D00016A127A130A5C8011A2F0B2F0E94602104
:1059E000F801E052F64F808391831A2F0B2F0E940B
:1059F000AF21BB2319F40A2F0E946D3A01E00093F6
:105A0000E50C9CC22CE636E08E010E941C1E002391
:105A100041F42AE636E08E010E941C1E002309F4A0
:105A200043C1BE01605F7F4FE9E7FEE930E08B01D3
:105A300048E150E00E94B24E923071F4FE01FF96B0
:105A400005A116A127A130A5073040E0140740E0CA
:105A5000240740E0340720F002E00E94A2206EC23A
:105A600001E00093E50CFE01FF9605A116A127A118
:105A700030A5102F07E00E94412040E452EE60E084
:105A800070E080E03AC002E0809F8001212F220F69
:105A9000220B322F040F151F261F371F0F5F1F4FBA
:105AA0002F4F3F4FF801322F3BBF069000E00BBF56
:105AB000302C222402E0809F8001212F220F220B14
:105AC000322F040F151F261F371FF801322F3BBF3F
:105AD0000690202D00E00BBF30E0220D331D2F7FFC
:105AE0003370FE01E55CFE4F082F10E0000F111F20
:105AF000E00FF11F2083318383958F3120F2FE0167
:105B0000FF9605A116A127A130A540E450E00E9410
:105B1000114E005C1F4F80E026C022E0829F000EE5
:105B2000111E21E0020E20E0121EF001E052F64F9D
:105B3000508140E022E0829F000E111EF001E052F1
:105B4000F64F208130E0240F351F2F7F3370FE0188
:105B5000E350FF4F482F50E0440F551FE40FF51F4F
:105B60002083318383958F31C0F280E068C0FE01CD
:105B7000E55CFE4F082F10E0000F111FE00FF11F32
:105B8000208131812F7F33708E0103501F4FFE0122
:105B9000709690E0E80FF91F408150E0440F551FC8
:105BA000040F151FE02FF12F008111810F7F13705B
:105BB000201B310B8E01055C1E4FFE01709690E09C
:105BC000E80FF91F408150E0440F551F040F151FC7
:105BD000E02FF12F008111810F7F1370020F131F2F
:105BE00022E0829F20E0020E22E0121EF001E0522D
:105BF000F64F008311838E0103501F4FFE017096F4
:105C000090E0E80FF91F208130E0220F331F020FD0
:105C1000131FE02FF12F0081118100701C7F22E003
:105C2000829F20E0020E22E0121EF001E052F64FA9
:105C300020813181202B312B2083318383958F313B
:105C400038F590E0FC01EB58F64F00810023B1F3EA
:105C5000FE01709690E0E80FF91F00810F3F09F0F8
:105C600086CFFE01E350FF4F082F10E0000F111FF9
:105C7000E00FF11F0081118122E0829F20E0020EDF
:105C800022E0121EF001E052F64F00831183D6CFBE
:105C900007E00E94742080E08F3108F04FC1082F88
:105CA0000E946D3A8395F8CF26E636E08E010E9479
:105CB0001C1E0023C1F000E00E94A2200E94170FCA
:105CC000093519F0093709F039C10E9493220E9461
:105CD0001823A0E0BA2F1A2F0B2F0E94C62001E034
:105CE0000093E50C2BC121E636E08E010E941C1EBC
:105CF000002341F42DE536E08E010E941C1E002396
:105D000009F418C110E088242FEF3FE0A9010E9498
:105D1000F34D22EF3FE0A9010E94FF4D01E12FEF7B
:105D20003FE0A9010E94FF4D80E090E006C0FC0129
:105D3000E052F64F0081100F0196803002E090078C
:105D4000B0F30091FF09011B0A950093FF090EE2D1
:105D50000E94E60D80E090E00BC0FC01E052F64F9F
:105D600000819C012050384FA9010E94FF4D0196EF
:105D7000803002E0900788F300911E0C20E03AE0AA
:105D8000A9010E94FF4D00911F0C21E03AE0A901FA
:105D90000E94FF4D80E090E001C00196803002E05B
:105DA000900770F49C012050384FA9010E94F34DD8
:105DB000FC01E052F64F1081011779F38824839497
:105DC000E3EEFCE00081118125EF3FE0A9010E9494
:105DD000FF4D882009F075C025EF3FE0A9010E9422
:105DE000F34DE3EEFCE020813181021709F069C038
:105DF0000AEA24EF3FE0A9010E94FF4D08E001BD3F
:105E000004EF11E00E94670C25EF3FE0A9010E941A
:105E1000F34D10E0E3EEFCE000831183E3EEFCE0E1
:105E2000008111810F7F10700083118388240FEF90
:105E300024EF3FE0A9010E94FF4DE3EEFCE000816A
:105E4000118120E030E040E052E060E070E00E942C
:105E5000524E2801390100E0400E00EE501E00E0D5
:105E6000601E00E0701E80E090E001C0019680306E
:105E700002E09007C0F49C012050384FA9010E9415
:105E8000F34D602F8C0120E030E0040D151D261D20
:105E9000371DF801322F3BBF069000E00BBF6015A5
:105EA00029F302E0802E20E03AE0A9010E94F34DA0
:105EB00000931E0C21E03AE0A9010E94F34D0093EB
:105EC0001F0C8820F9F40E94FB210091F5090023A2
:105ED00061F0E3EEFCE0008111812091F50930E0F2
:105EE00020503F4FA9010E94FF4D0EE215E10E9494
:105EF0005B4C0E941823A0E0BA2F1A2F0B2F0E9490
:105F0000C62009C005ED1DE00E945B4C00E3800E39
:105F1000082D0E94E60D00E00093E50C22EF3FE023
:105F2000A9010E94F34D2FEF3FE0A9010E94FF4D10
:105F3000AD9804C008EE1DE00E945B4C0091F4098E
:105F4000091599F00091F409013F20F000E0009359
:105F5000F40907C00091F409083018F007E0009335
:105F6000F4090E940F219090F4091A2F0B2F0E9420
:105F7000D1220C94C7249A938A93802F082F0E94D1
:105F8000AA4D0F3F2FEF120719F400E012E01CC0DA
:105F9000E3EEFCE020813181232B51F090E0880F6B
:105FA000991FFC01E056F64F20813181021B130B33
:105FB000212F27FF03C000E010E006C0003024E0DE
:105FC000120710F00FEF13E08991999108959A93B9
:105FD0008A93902F812F02E00E94E60D0BE10E9430
:105FE000E60D0BE50E94E60D8A3038F0082F4AE0F6
:105FF0000E94034E005D0E94E60D082F4AE00E94B9
:10600000034E042F005D0E94E60D0BE30E94E60D97
:106010009A3038F0092F4AE00E94034E005D0E943A
:10602000E60D092F4AE00E94034E042F005D0E94F6
:10603000E60D06E60E94E60D8991999108959A93DE
:106040008A93FA93EA933A922A921A920A927A934C
:106050006A935A934A933A932A931A930A938FB75F
:106060009BB700E00BBF78940091E80C002349F047
:106070000091E70C002321F004E20E94E60D01C02C
:10608000CED0EAEFFCE0008111810F5F1F4F00834B
:1060900011830091260E102F13951093260E0F706A
:1060A000002309F06EC0ECEFFCE000811181012BB0
:1060B00041F0ECEFFCE000811181015010400083C1
:1060C00011830091F90C002349F0E9EFFCE0008115
:1060D0000A95008308E015B3102715BBAA9AA99A60
:1060E00024B135B10091E70D10E003701070000F7E
:1060F000111FF801E152F24F20833183E7EEFDE0FA
:10610000008103950083037007B90091270E102FBB
:1061100013951093270E0770002399F5E6EDFDE027
:106120000081039500830E940A44879B2AC0969BA6
:1061300028C00091F30C002321F500919A000F77FD
:1061400000939A00959A96980FE113E00150104041
:10615000E9F700C0000000919B00102F17FF0AC054
:1061600000919C00053531F404E110E00E94670CB9
:1061700008E001BD969A959800919A0000680093F6
:106180009A00E8EEFDE0008107FF0CC00091260EAA
:10619000002311F4A89815C00091260E083089F448
:1061A000A89A0FC00091260E1091E80D102311231C
:1061B00041F40091E80D002321F001E015B3102710
:1061C00015BB00E000931B0D9BBF8FBF0991199178
:1061D0002991399149915991699179910990199031
:1061E00029903990E991F9918991999118959A930B
:1061F0008A93C80120E030E010E20EEF0E94C84D03
:10620000E5EFFCE08083918301E00093F40C0093C0
:10621000E80C00E00093E60C8991999108950E94A2
:10622000C54E24970091F40C002309F44DC000E002
:106230000093691000E010E0EFE5F0E100831183C6
:10624000EDE5F0E100831183E1E6F0E100831183E5
:1062500000E00093B00C03E000936710CC2431C041
:1062600002E0C09E800100501E4FF801E052F64F40
:10627000208131810C2D10E0000F111FF801EC5C22
:10628000F04F2083318300E010E02C2D30E0220F0E
:10629000331FF901E650F04F008311832C2D30E0BD
:1062A000220F331FF901E45DF14F008311832C2D80
:1062B00030E0220F331FF901E854F04F00831183BF
:1062C000C3940FE1C01660F2EDE5F0E100811181A9
:1062D000EFE5F0E1208131810217130708F00CC3CC
:1062E000EDE5F0E1008111810F5F1F4F0083118305
:1062F000E2EEFCE0008100FF86C0EAEFFCE00081F6
:1063000011810370002309F059C002E20093A00735
:1063100003E00093A10722E012E006E60E94374B5B
:10632000002331F000912708109128089091290846
:1063300000916A10000F00936A10EAE6F0E1008114
:1063400001FF08C09B3068F0EAE6F0E100810160DF
:10635000008307C0933328F0EAE6F0E10081016092
:10636000008302E20093A00703E00093A10722E06C
:1063700012E005E60E94374B002331F00091270818
:10638000109128088091290800916B10000F00934C
:106390006B10EBE6F0E1008101FF08C08B3098F153
:1063A000EBE6F0E10081016000832DC0833358F1FA
:1063B000EBE6F0E100810160008325C0EAEFFCE03C
:1063C000008111810370013061F408E20093A0079D
:1063D00004E00093A10722E012E007E60E94374B99
:1063E00012C0EAEFFCE0008111810370023059F421
:1063F00004E30093A00704E00093A10722E012E069
:1064000007E60E94374B00916710033009F474C20D
:1064100080E00CE190E0FC01E056F84F00838395AA
:1064200004E090E0FC01E056F84F00838395CC2413
:106430004CC001E010E02C2D30E0205E3F4FF90110
:10644000EF55F34F408142954F700E94214E90E0EE
:10645000FC01E056F84F0083839501E010E02C2DFD
:1064600030E0205E3F4FF901EF55F34F40814F7010
:106470000E94214E90E0FC01E056F84F0083839586
:1064800002E0C09E00E0000E02E0101EF001E052AB
:10649000F64F0081118190E0FC01E056F84F008337
:1064A000839502E0C09E00E0000E02E0101EF001A5
:1064B000E052F64F00811181012F10E090E0FC01C5
:1064C000E056F84F00838395C3940FE1C01608F09F
:1064D0000EC2DD24F601EB58F64F00810023A1F334
:1064E00000916710002309F092C00C2D10E0000FFE
:1064F000111FF801EA58F04F008111812C2D30E076
:10650000220F331FF901E854F04F20813181021B23
:10651000130B212F220F220B322FEDE5F0E14081EA
:10652000518160E070E00E94524EEFE5F0E1408161
:10653000518160E070E00E949C4E2C2D30E0220FD3
:10654000331FF901E854F04F40815181400F511F32
:106550002C2D30E0220F331FF901E650F04F40831D
:1065600051832C2D30E0220F331FF901E854F04FF6
:106570002081318115950795020F131F212F220FBE
:10658000220B322FEDE5F0E14081518160E070E0B7
:106590000E94524E40E950E060E070E00E94524E8E
:1065A0004FE050E060E070E00E949C4E012F122FFF
:1065B000232F330F330B2595179507952C2D30E09E
:1065C000220F331FF901E055F14F008311830C2D89
:1065D00010E0000F111FF801EE50F14F20813181C2
:1065E0000C2D10E0000F111FF801E055F14F008154
:1065F0001181020F131F22E0C29E20E0020E22E052
:10660000121EF001E052F64F0083118310C1009179
:106610006710013009F046C00C2D10E0000F111F6B
:10662000F801EE50F14FA081B1810C2D10E0000F68
:10663000111FF801E259F14F00811181212F220F22
:10664000220B322FEDE5F0E14081518160E070E0F6
:106650000E94524EEFE5F0E14081518160E070E030
:106660000E949C4E0A0F1B1F22E0C29E20E0020ED9
:1066700022E0121EF001E052F64F008311830C2D30
:1066800010E0000F111FF801EA58F04F208131810E
:106690000C2D10E0000F111FF801E650F04F208381
:1066A0003183C5C0DD24F601E45CFF4E0081002388
:1066B00009F078C00C2D10E0000F111FF801E8540C
:1066C000F04F00811181119501951040212F220F6B
:1066D000220B322FEDE5F0E14081518160E070E066
:1066E0000E94524EEFE5F0E14081518160E070E0A0
:1066F0000E949C4E2C2D30E0220F331FF901E854EC
:10670000F04F40815181400F511F2C2D30E0220F5E
:10671000331FF901E650F04F408351832C2D30E0B8
:10672000220F331FF901EE50F14FA081B1812C2DC2
:1067300030E0220F331FF901E854F04F20813181FE
:1067400015950795020F131F212F220F220B322FB1
:10675000EDE5F0E14081518160E070E00E94524E31
:1067600040E950E060E070E00E94524E4FE050E09F
:1067700060E070E00E949C4E012F122F232F330FF8
:10678000330B2595179507950A0F1B1F22E0C29E14
:1067900020E0020E22E0121EF001E052F64F0083CC
:1067A000118345C00C2D10E0000F111FF801EE50B1
:1067B000F14FA081B1810C2D10E0000F111FF801E5
:1067C000E259F14F00811181212F220F220B322F2C
:1067D000EDE5F0E14081518160E070E00E94524EB1
:1067E000EFE5F0E14081518160E070E00E949C4E55
:1067F0000A0F1B1F22E0C29E20E0020E22E0121EA2
:10680000F001E052F64F008311830C2D10E0000FD1
:10681000111FF801EA58F04F208131810C2D10E052
:10682000000F111FF801E650F04F2083318302E082
:10683000C09E00E0000E02E0101EF001E052F64F94
:10684000018107FF0EC000E010E022E0C29E20E0C0
:10685000020E22E0121EF001E052F64F0083118377
:106860001CC002E0C09E00E0000E02E0101EF0011D
:10687000E052F64F20813181203004E0300768F08B
:106880000FEF13E022E0C29E20E0020E22E0121E73
:10689000F001E052F64F0083118390E0FC01E056D6
:1068A000F84FC0828395E2EEFCE0008100FFC1CD8D
:1068B00000916A100F3F19F004E1C01649F00091F1
:1068C0006B100F3F09F4B5CD05E1C01609F0B1CD4D
:1068D00000E890E0FC01E056F84F0083839500E863
:1068E00090E0FC01E056F84F00838395C9CD282F36
:1068F00013E80EEF0E94BC4A00916910002321F0BA
:1069000000E00093E80CE5C5EDE5F0E100811181C0
:10691000EFE5F0E1208131810217130708F4D9C5B2
:1069200000E010E0EDE5F0E100831183CC2427C006
:1069300002E0C09E00E0000E02E0101EF001E052F6
:10694000F64F208131810C2D10E0000F111FF8014E
:10695000EE50F14F208331830C2D10E0000F111FFA
:10696000F801E650F04F208131810C2D10E0000F2E
:10697000111FF801E854F04F20833183C3940FE1D5
:10698000C016B0F200916710002309F09FC001E02B
:1069900000936710E3E6F0E100811181E5E6F0E1A4
:1069A00020813181220F331F021B130BEFE5F0E131
:1069B00000831183CC2446C00C2D10E0000F111F62
:1069C000F801E45DF14F808191810C2D10E0000F02
:1069D000111FF801E055F14F00811181801B910BCF
:1069E0000C2D10E0000F111FF801EA58F04F008144
:1069F0001181212F220F220B322FE5E6F0E1408199
:106A0000518160E070E00E94524E4CE050E060E046
:106A100070E00E94524E45E050E060E070E00E945D
:106A20009C4E012F122F232F330F330B801B910B02
:106A30000C2D10E0000F111FF801E259F14F808377
:106A40009183C3940FE1C01608F0D6C0DD24F6018F
:106A5000E45CFF4E0081013009F0AECF0C2D10E058
:106A6000000F111FF801E45DF14F008111812C2D01
:106A700030E0220F331FF901E055F14F20813181C1
:106A8000021B130B212F220F220B322FEFE5F0E117
:106A90004081518160E070E00E94524EE3E6F0E1F7
:106AA00040815181E5E6F0E160817181461B570B21
:106AB00060E070E00E949C4E2C2D30E0220F331FCE
:106AC000F901E259F14F00831183BBCF00916710A8
:106AD0000130D1F502E000936710E5E6F0E10081B6
:106AE0001181EFE5F0E100831183CC240FE1C016A2
:106AF00008F082C00C2D10E0000F111FF801E45DBA
:106B0000F14F208131810C2D10E0000F111FF80191
:106B1000E259F14F00811181201B310B0C2D10E047
:106B2000000F111FF801E055F14F00811181201B6A
:106B3000310B0C2D10E0000F111FF801E259F14F3D
:106B400020833183C394D2CF009167100230B1F417
:106B5000E1E6F0E100811181012B61F003E0009397
:106B60006710E1E6F0E100811181EFE5F0E10083DB
:106B7000118342C000E0009367103EC0009167108F
:106B80000330D1F5CC2432C002E0C09E00E0000EFC
:106B900002E0101EF001E052F64F208131810C2DF1
:106BA00010E0000F111FF801EC5CF04F20833183DF
:106BB00000E010E02C2D30E0220F331FF901E650E9
:106BC000F04F008311832C2D30E0220F331FF90189
:106BD000E45DF14F008311832C2D30E0220F331F31
:106BE000F901E854F04F00831183C3940FE1C016FC
:106BF00058F200E00093671000916710002309F03D
:106C000068C4E8E6F0E10081039500830091681014
:106C10001091B50C011728F40091F40C002309F42D
:106C2000DFC00091F40C002399F5E5EFFCE0008152
:106C30001181E7EFFCE0008311830091B00C002389
:106C400029F0E1EAFCE007850A9507870091B00C7E
:106C50000023F1F40091E60C013039F400E010E07B
:106C6000E5EFFCE00083118313C00091E60C0230D5
:106C700041F40091BB0C10E0E5EFFCE000831183D0
:106C800007C00091BA0C10E0E5EFFCE0008311832F
:106C9000E5EFFCE000811181012B21F401E000937C
:106CA00069109EC000E00093F40CE3EEFCE000816C
:106CB0001181E5EFFCE0208131810217130741F5D6
:106CC00000E010E020E030E0E8E2FEE00083118325
:106CD000228333830091B00C002309F053C0ADE050
:106CE000B0E0A03400E0B00708F04CC0E8E2FEE0FD
:106CF00000811181228133810A0F1B1FF801E052AC
:106D0000F64F0081FD01EF55F34F00831196E9CF57
:106D1000E5EFFCE00081118120E030E0322F212FEF
:106D2000102F00E0110F221F331F005010422F4F71
:106D30003F4FE8E2FEE0008311832283338300911A
:106D4000B00C0023F9F4ADE0B0E018C0E8E2FEE0DA
:106D500040815181628173818D0120E030E0040F18
:106D6000151F261F371FF801322F3BBF069000E08A
:106D70000BBFFD01EF55F34F00821196A03400E0E8
:106D8000B00720F3E8E2FEE0008111812281338127
:106D9000005C1F4F2F4F3F4F0083118322833383AB
:106DA0000091B50C083020F40091B50C002381F45B
:106DB0000BE01DE00E945B4CE5EFFCE000811181DF
:106DC0000E94ED0E0DE50E94E60D01E000936910B2
:106DD0000091B00C002309F428CF00E00093681064
:106DE000A0E0B0E020C0E8E2FEE000811181228155
:106DF0003381A801B9014F5F5F4F6F4F7F4FE8E2CA
:106E0000FEE04083518362837383F801322F3BBFDE
:106E1000069000E00BBF8D01005C1D4FF801E052B1
:106E2000F64F00821196A03400E0B00758F5E3EE6B
:106E3000FCE000811181E5EFFCE020813181021747
:106E4000130789F6E8E2FEE0008111812281338197
:106E5000F801E052F64F20818D01005C1D4FF801D2
:106E6000E052F64F2083E8E2FEE0008111812281AA
:106E700033810F5F1F4F2F4F3F4F008311832283BA
:106E80003383D0CF009168100395E5EFFCE080815B
:106E900091811091B50C011708F459C00091E60CCE
:106EA000013039F400E010E0E5EFFCE000831183ED
:106EB00015C00091E60C023031F400E00093B00CF4
:106EC0008091BB0C0BC00091B00C023028F0E5EFB4
:106ED000FCE08081918102C08091BA0C90E0E3EEE9
:106EE000FCE0008111818017910759F400E410E063
:106EF00020E030E0E8E2FEE0008311832283338368
:106F000026C0882379F4E8E2FEE000811181228125
:106F1000338100541040204030400083118322838D
:106F2000338315C0082F10E020E030E0322F212FEE
:106F3000102F00E0110F221F331F005C1F412F4F45
:106F40003F4FE8E2FEE00083118322833383A0E019
:106F5000B0E01BC0E8E2FEE04081518162817381B4
:106F60008D0120E030E0040F151F261F371FF801A8
:106F7000322F3BBF069000E00BBF8D0100581D4F24
:106F8000F801E052F64F00821196A03400E0B007FD
:106F9000D0F4E3EEFCE0008111818017D9F6E8E23D
:106FA000FEE000811181228133810A0F1B1FF8014D
:106FB000E052F64F20818D0100581D4FF801E0523C
:106FC000F64F2083E1CF00916910002309F081C2C0
:106FD00000915E0C10E045E00E94214E4091B70CFC
:106FE00050E00E942D4EE1E6F0E100831183009114
:106FF0005F0C1091B70C019F800145E00E94274E65
:10700000D8010A2F0B2B11F4A1E0B0E020E030E012
:10701000CC240EC00C2D10E0000F111FF801E45D10
:10702000F14F008111812017310708F49801C394B2
:107030000FE1C01608F0FCC0DD24F601EB58F64F56
:1070400000810023A1F30C2D10E0000F111FF801A7
:10705000EC5CF04F4081518102E0C09E00E0000EE8
:1070600002E0101EF001E052F64F408351830C2DD8
:1070700010E0000F111FF801EE50F14F40835183D3
:1070800000E010E04C2D50E0440F551FFA01E05590
:10709000F14F0083118302E0C09E00E4000E02E085
:1070A000101EF001E052F64F008111814C2D50E08E
:1070B000440F551FFA01E056F64F60817181DD24BF
:1070C000F601E954F24F4081542F550F550B460FEE
:1070D000571F040F151F412F47FF03C000E010E0AA
:1070E00006C0003044E0140710F00FEF13E04C2D01
:1070F00050E0440F551FFA01EC5CF04F4081518184
:10710000B801641B750B4C2D50E0440F551FFA015C
:10711000E45DF14F608371834C2D50E0440F551FA7
:10712000FA01EC5CF04F608171814C2D50E0440F0E
:10713000551FFA01EC5CF04F0083118342E0C49EBE
:1071400040E8040E42E0141EF001E052F64F2080A9
:1071500031804C2D50E0440F551FFA01E056F64F98
:1071600000801180020C131CDD24F601E954F24F5B
:107170004081542F550F550B400D511D052E07FE14
:1071800003C040E050E006C04030E4E05E0710F08D
:107190004FEF53E06017710718F40417150730F02C
:1071A0000617170728F44017510710F400E001C034
:1071B00001E0002391F4E1E6F0E100811181012B6F
:1071C00061F40091681010E0E091B50CF0E03197A7
:1071D0000E171F074CF0882339F400E0DD24F60178
:1071E000E45CFF4E008306C001E0DD24F601E45CB0
:1071F000FF4E00830091B10C0A3009F418CF0C2D1A
:1072000010E0000F111FF801E45DF14F4081518142
:1072100055230AF0FFCE0C2D10E0000F111FF801CE
:10722000E45DF14F00811181119501951040FBCE75
:107230000091B10C0A3029F4E3E6F0E1A083B183B8
:1072400013C0890148E250E00E94114EC8018D012F
:1072500043E050E00E94114EA8018C010E942D4E87
:10726000E3E6F0E1008311830091B90C10E0E5E65C
:10727000F0E100831183E5E6F0E100811181000F68
:10728000111FE3E6F0E12081318102171307E8F1D5
:10729000E2E7F9E0008102FF13C00BE50E94E60D72
:1072A000009168100E94CF0D0CE20E94E60DE3E60B
:1072B000F0E1008111810E94ED0E0DE50E94E60DC6
:1072C000E3E6F0E100811181012B39F400E010E0E8
:1072D000E5E6F0E10083118318C0E3E6F0E1008108
:1072E00011810150104016950795E5E6F0E1008305
:1072F0001183E5E6F0E100811181012B31F400E01A
:1073000010E0E3E6F0E100831183E3E6F0E10081C1
:10731000118120E030E0000F111F221F331FE5E62E
:10732000F0E180819181A0E0B0E0880F991FAA1F51
:10733000BB1F081B190B2A0B3B0B48015901880C7A
:10734000991CAA1CBB1C880E991EAA1EBB1E000FEE
:10735000111F221F331F088319832A833B83082DA3
:1073600009290A290B2929F49924AA24BB24882451
:107370008394088119812A813B81012B022B032BE5
:1073800041F401E010E020E030E0088319832A8313
:107390003B83CC2442C00419150926093709A401EE
:1073A000B5010E949C4E2C2D30E0220F331FF901B5
:1073B000EA58F04F008311830C2D10E0000F111FCD
:1073C000F801EA58F04F20813181203004E0300785
:1073D0005CF00FEF13E02C2D30E0220F331FF9018A
:1073E000EA58F04F008311830C2D10E0000F111F9D
:1073F000F801EA58F04F2081318121300CEF30073D
:107400005CF401E01CEF2C2D30E0220F331FF9015A
:10741000EA58F04F00831183C3940FE1C01608F0BF
:1074200050C00C2D10E0000F111FF801E854F04F70
:1074300000811181212F220F220B322FAC01BD01BF
:107440000E94524E280139010C2D10E0000F111F2F
:10745000F801E45DF14F00811181212F220F220BF1
:10746000322F0801190140E05AE060E070E080012D
:1074700091010E94524E080119014CE050E060E079
:1074800070E0800191010E949C4EDD24F601E45CD5
:10749000FF4E4081442309F07ECF041915092609C7
:1074A0003709488159816A817B810E949C4E2C2D2D
:1074B00030E0220F331FF901EA58F04F00831183A7
:1074C0007BCFE5E6F0E100811181EFE5F0E100839B
:1074D00011832496EEE00C94D64E0E94CF4E802F5E
:1074E00090E0FC01EB58F64F0081002309F47FC0C7
:1074F00002E0809F800100501E4FF801E052F64FDD
:10750000018105FF06C020E018E1082F0E94C04D50
:107510006EC0E3EEFCE000811181012BC9F002E0B6
:10752000809F00E0000E02E0101EF001E052F64FD6
:10753000008111810F7F1370282F30E0220F331F3D
:10754000F901E056F64FA081B181A00FB11F0DC027
:1075500002E0809F00E0000E02E0101EF001E05209
:10756000F64FA081B181AF7FB3700B2F07FF03C02F
:10757000A0E0B0E006C0A03004E0B00710F0AFEF2C
:10758000B3E014E2082F0E94AA4D98012F3F03E0B8
:10759000300758F4A217B30720F42A1B3B0B8901CC
:1075A00006C08D01021B130B02C008E010E0169507
:1075B000079516950795083020E0120710F408E0AB
:1075C00010E02EE12093A0072A2F2093A107AB2FD4
:1075D000B0E0A093A207202F2093A307012F10E073
:1075E0000093A40725E013E0082F0E94374BE4E046
:1075F0000C94E04E0E94CF4ED8010091E80C00237D
:1076000009F041C00A2F0B2BF1F1A03800E0B007C0
:10761000D0F500E010E0E3EEFCE00083118380E0B1
:107620000BC022E0829F900120503E4FF901E052B2
:10763000F64F0083118383958F3110F590E0FC01A4
:10764000EB58F64F00810023B1F318E1082F0E9498
:107650009B4D013029F41EE1082F0E94BB2F04C06E
:1076600014E2082F0E94BB2F003020E41207C9F655
:107670000DED1DE00E945B4C082F0E94CF0DDBCF6B
:107680008D010E94F730E4E00C94E04E6AC00E9445
:10769000170F1091FF0C163018F010E01093FF0C2C
:1076A0002091FF0C30E0F901E050F34F0083EFEF41
:1076B000FCE0108113951083053551F50091FF0C06
:1076C0000250073008F00A5F10E0F801E050F34F75
:1076D00000810F3FE9F400E00093FF0C0FEF2091D1
:1076E000FF0C30E0F901E050F34F0083EFEFFCE0D6
:1076F00000810395008305E52091FF0C30E0F9013E
:10770000E050F34F0083EFEFFCE00081039500832E
:107710000091FF0C063029F50091000D0F3F09F58F
:107720000091010D0535E9F40091020D1091030D52
:1077300010950117B1F40091040D1091050D1095ED
:10774000011779F401E00093FE0C3091040D20E064
:107750000091020D10E0020F131FE9EEFCE0008320
:1077600011830091090D1091080D011709F08FCFB9
:1077700008959A938A93C901083C09F0CFC0183143
:1077800051F4082F092B21F402E00093E60C01C10B
:107790008C0130DFFEC01A3111F01B3149F5EBEEE0
:1077A000FCE0808391830FEF0E94E60D05E50E94C7
:1077B000E60DEBEEFCE0008111810E94E60DEBEEA0
:1077C000FCE00081118100950E94E60DEBEEFCE0EB
:1077D00000811181012F10E00E94E60DEBEEFCE02C
:1077E00000811181012F10E000950E94E60DD1C0AB
:1077F0001F3159F4882311F401E001C000E0102F7B
:1078000010FDAB9A10FFAB98C4C01232A1F540E056
:1078100050E010E020E030E000E00E94BC0C0023CB
:1078200009F4B7C0EFEEFCE00081118108171907D9
:1078300039F040E050E010E09C0101E00E94BC0CF7
:10784000E2E6F9E0038114810817190709F4A1C0E1
:10785000E2E6F9E083839483082F23E030E0A90176
:107860000E94FF4D892F90E0082F24E030E0A9010D
:107870000E94FF4D8EC0113229F4ECEFFCE08083B2
:10788000918387C0153221F48C010E94670E81C05C
:10789000163251F48C010E94670E0DE00E94E60D35
:1078A0000AE00E94E60D75C01832A1F540E050E0F4
:1078B00010E020E030E000E00E94BC0C002309F45E
:1078C00068C0E1EFFCE0008111810817190739F069
:1078D000AC0110E020E030E004E00E94BC0CE2E6E5
:1078E000F9E0018512850817190709F452C0E2E68C
:1078F000F9E081879287082F29E030E0A9010E94F2
:10790000FF4D892F90E0082F2AE030E0A9010E9466
:10791000FF4D3FC002E010E8E0D43BC00436F0F079
:107920000D36E0F42091E80C222339F021E0209379
:107930001B0D20911B0D2223E1F7E2E5F7E1212F3A
:1079400030E0E20FF31F2491223021F49C010E94C9
:10795000C84D1FC0282F0E94C04D1BC02091E80CAD
:10796000222339F021E020931B0D20911B0D2223AF
:10797000E1F7EAE1F7E1212F30E0E20FF31F249174
:10798000223021F49C010E94C84D03C0282F0E9480
:10799000C04D899199910895083C09F0E4C01831CF
:1079A00081F4E5EFFCE000811181012B29F4E7EF80
:1079B000FCE0008111810895E5EFFCE00081118178
:1079C0000895193121F40091E80C10E008951A315E
:1079D00011F01B3129F4EBEEFCE0008111810895D8
:1079E0001C3111F01D3149F451DE00E00093FE0C12
:1079F000E9EEFCE00081118108951E3129F446DE94
:107A00000091FE0C10E008951F3141F405B3069576
:107A1000069506950095017010E008951232B1F5B3
:107A200040E050E010E020E030E000E00E94BC0CBC
:107A3000002339F1E2E6F9E003811481EFEEFCE086
:107A40002081318102171307E1F0EFEEFCE00081A5
:107A50001181E2E6F9E003831483EFEEFCE000819C
:107A6000118123E030E0A9010E94FF4DEFEEFCE020
:107A700000811181012F10E024E030E0A9010E9473
:107A8000FF4DE2E6F9E0038114810895143269F4B0
:107A900040E050E010E020E030E000E00E94BC0C4C
:107AA000EDEEFCE00081118108951032B9F400E0A0
:107AB000809902C0006111E00C9902C0086011E0D9
:107AC0000D9902C0046011E00E9902C0026011E03D
:107AD0000F9902C0016011E010E00895113229F4FD
:107AE000ECEFFCE00081118108951832B1F540E01F
:107AF00050E010E020E030E000E00E94BC0C0023E9
:107B000039F1E2E6F9E001851285E1EFFCE0208140
:107B1000318102171307E1F0E1EFFCE000811181F0
:107B2000E2E6F9E001871287E1EFFCE000811181D4
:107B300029E030E0A9010E94FF4DE1EFFCE0008167
:107B40001181012F10E02AE030E0A9010E94FF4DD1
:107B5000E2E6F9E001851285089501E010E8BDD361
:107B60000FEF1FEF08950436E8F00E36D8F4209199
:107B7000E80C222339F021E020931B0D20911B0DEE
:107B80002223E1F7E2E5F7E1212F30E0E20FF31FD6
:107B90002491223019F40E94AA4D08950E949B4D11
:107BA00010E008950F31D8F42091E80C222339F029
:107BB00021E020931B0D20911B0D2223E1F7EAE128
:107BC000F7E1212F30E0E20FF31F2491223019F466
:107BD0000E94AA4D08950E949B4D10E008952091A7
:107BE000E80C222339F021E020931B0D20911B0D7E
:107BF0002223E1F70E94AA4D08959A938A93ECE11B
:107C0000FDE00081118198012F5F3F4FECE1FDE025
:107C10002083318320E030E0005010462F4F3F4F4B
:107C2000F801322F3BBF0690002D10E01BBFECE1A6
:107C3000FDE0408151819A012F5F3F4FECE1FDE073
:107C40002083318360E070E0405050466F4F7F4F9B
:107C5000FA01362F3BBF0690202D10E01BBFECE150
:107C6000FDE040815181CA010196ECE1FDE0808395
:107C7000918360E070E0405050466F4F7F4FFA01B3
:107C8000362F3BBF069010E01BBF002321F4102DC0
:107C9000022F82DE4EC0023061F4102D30E0220F40
:107CA000331FF901E85DF24F20813181022F74DE2C
:107CB00040C0013069F4002D10E0000F111FF801E1
:107CC000E85DF24F00811181102F022F65DE31C077
:107CD0000330A9F4002D10E0000F111FF801E85D3A
:107CE000F24F00811181102F30E0220F331FF90174
:107CF000E85DF24F20813181022F4EDE1AC0043040
:107D000039F4502D40E0022F10E0040F151F11C070
:107D1000053069F4102D00E030E0200F311F220FF4
:107D2000331FF901E85DF24F0081118102C000E0CC
:107D300010E08991999108950E94CF4EA801ECE13D
:107D4000FDE00081118198012F5F3F4FECE1FDE0E4
:107D50002083318320E030E0005010462F4F3F4F0A
:107D6000F801322F3BBF0690002D10E01BBFECE165
:107D7000FDE000801180C0010196ECE1FDE0808310
:107D80009183C001A0E0B0E080509046AF4FBF4F5C
:107D9000FC013A2F3BBF0690602D10E01BBFECE1C9
:107DA000FDE000801180C0010196ECE1FDE08083E0
:107DB0009183C001A0E0B0E080509046AF4FBF4F2C
:107DC000FC013A2F3BBF069010E01BBF002329F4B3
:107DD0009A01102D062FCDDC4BC0023069F49A01B8
:107DE000102D70E0660F771FFB01E85DF24F4081B8
:107DF0005181042FBEDC3CC0013071F49A01002D8A
:107E000010E0000F111FF801E85DF24F00811181B1
:107E1000102F062FAEDC2CC00330B1F49A01002DD8
:107E200010E0000F111FF801E85DF24F0081118191
:107E3000102F70E0660F771FFB01E85DF24F408165
:107E40005181042F96DC14C0043021F407E010E0C7
:107E500044D20EC0053061F4102D00E070E0600FD8
:107E6000711F660F771FFB01E85DF24F408351835E
:107E7000E4E00C94E04EC1DEEEE1FDE0008311830E
:107E8000ECE1FDE00081118198012F5F3F4FECE1B3
:107E9000FDE02083318320E030E0005010462F4F7A
:107EA0003F4FF801322F3BBF069000E00BBF00921E
:107EB000240DA3DEE0E2FDE0008311830091240D98
:107EC000002379F4EEE1FDE000811181E0E2FDE0C4
:107ED000208131810217130711F401E0089500E0B9
:107EE00008950091240D013079F4E0E2FDE0008175
:107EF0001181EEE1FDE0208131810217130710F4BA
:107F000001E0089500E008950091240D023079F415
:107F1000EEE1FDE000811181E0E2FDE020813181B0
:107F20000217130710F001E0089500E00895009192
:107F3000240D033079F4EEE1FDE000811181E0E2EF
:107F4000FDE0208131810217130710F401E008954C
:107F500000E008950091240D043079F4E0E2FDE0A2
:107F600000811181EEE1FDE02081318102171307CC
:107F700010F001E0089500E008950091240D05300F
:107F800079F4EEE1FDE000811181E0E2FDE0208185
:107F900031810217130711F001E0089500E0089500
:107FA00005E010E09AD100E008950091250D013020
:107FB00061F40091270D002331F00091260D00237C
:107FC00011F001E0089500E008950091250D0230C0
:107FD00061F40091270D002321F40091260D002368
:107FE00011F001E0089500E0089506E010E075D179
:107FF00000E008959A938A930230C9F0ECE1FDE025
:10800000408151819A012F5F3F4FECE1FDE02083D9
:10801000318360E070E0405050466F4F7F4FFA016F
:10802000362F3BBF069010E01BBF0092230D10912E
:10803000230D1F5F09F440C1125091F01A9509F108
:108040001A9509F44CC01A9509F4F2C01A9509F46E
:10805000FBC01A9509F407C11A9509F41CC137C170
:10806000002331F0CADDECE1FDE00083118332C171
:10807000ECE1FDE0008111810D5F1F4F0083118352
:1080800029C1002319F1ECE1FDE0008111810D5FB0
:108090001F4F00831183B1DDE0E2FDE00083118317
:1080A000ECE1FDE000811181065010400083118356
:1080B000E0E2FDE0008111813FDEECE1FDE00081C6
:1080C00011810D5F1F4F0083118304C1ECE1FDE0BE
:1080D000008111810A5F1F4F00831183FBC00023C1
:1080E00009F49DC0ECE1FDE0008111810D5F1F4F9F
:1080F0000083118382DDEEE1FDE000831183ECE17A
:10810000FDE00081118198012F5F3F4FECE1FDE020
:108110002083318320E030E0005010462F4F3F4F46
:10812000F801322F3BBF069000E00BBF0092240DF8
:1081300064DDE0E2FDE0008311830091240D002363
:1081400059F4EEE1FDE000811181E0E2FDE0808183
:108150009181800F911F50C00091240D013059F47E
:10816000EEE1FDE080819181E0E2FDE0008111819E
:10817000801B910B41C00091240D023061F4EEE1AF
:10818000FDE000811181E0E2FDE0408151810E942B
:10819000114EC80131C00091240D033061F4EEE1AD
:1081A000FDE000811181E0E2FDE0408151810E940B
:1081B0002D4EC80121C00091240D003159F4EEE18B
:1081C000FDE000811181E0E2FDE08081918180236A
:1081D000912312C00091240D013159F4EEE1FDE02C
:1081E00000811181E0E2FDE080819181802B912B63
:1081F00003C004E010E071D0ECE1FDE000811181EA
:108200000A501040008311838C0196DDECE1FDE003
:1082100000811181095F1F4F008311835BC0ECE176
:10822000FDE000811181065F1F4F0083118352C062
:10823000002309F04FC0ECE1FDE000811181ECE189
:10824000FDE00083118346C0002321F00BE1009381
:10825000220D40C0ECE1FDE000811181ECE1FDE088
:108260000083118337C0002369F0ECE1FDE0008159
:1082700011810D5F1F4F7DD2C0DCECE1FDE000837A
:10828000118328C0ECE1FDE0008111810D5F1F4FDB
:10829000008311831FC0002331F095D2ECE1FDE093
:1082A0000083118317C0ECE1FDE000811181ECE156
:1082B000FDE0008311830EC0002361F4ECE1FDE0DA
:1082C00000811181ECE1FDE00083118303C003E133
:1082D00010E003D08991999108959A938A93C801E7
:1082E000E2E7F9E0008101FF1AC001E715E10E9411
:1082F0005B4C8C010E94ED0E0BE50E94E60DECE15B
:10830000FDE0008111810E94ED0E0AE30E94E60D5E
:108310000091230D0E94CF0D0DE50E94E60D89917D
:10832000999108950E94D04EA02FAA2311F49598F8
:10833000969A00E010E0ECE1FDE00083118380E01C
:1083400090E204E00093230DAA2321F002E315E15B
:108350000E945B4C00E00093220D05C002E04ADE63
:10836000AA2309F02FD10091220D0B3109F423C16A
:10837000ECE1FDE020813181203000EC300708F095
:108380001AC10091230D053009F415C1ECE1FDE09F
:10839000008111810817190708F00DC1ECE1FDE01B
:1083A0000081118198012F5F3F4FECE1FDE02083B8
:1083B000318320E030E0005010462F4F3F4FF8014E
:1083C000322F3BBF069000E00BBF0092230DE3E28B
:1083D000FDE0008107FFC2CF0091230D005849F056
:1083E0000A9509F46FC00A9509F4CCC00A95B1F159
:1083F000DEC041DD0093260D0091260D0093270D70
:10840000ECE1FDE00081118198012F5F3F4FECE12D
:10841000FDE02083318320E030E0005010462F4FF4
:108420003F4FF801322F3BBF069000E00BBF009298
:10843000250DAA2309F0C6D00091250D002309F0CF
:1084400092CF0091270DD6DDAA2309F48CCF00919D
:10845000270D002309F487CFB5D085CF0CDD00931D
:10846000260DA3DD0093270DECE1FDE000811181D5
:1084700098012F5F3F4FECE1FDE02083318320E046
:1084800030E0005010462F4F3F4FF801322F3BBFD6
:10849000069000E00BBF0092250DAA2309F092D0B0
:1084A0000091250D002309F05ECF0091270DA2DD7C
:1084B000AA2309F458CF0091270D002309F453CFC4
:1084C00081D051CF0091270D002339F1D4DC0093E6
:1084D000260DECE1FDE00081118198012F5F3F4FF7
:1084E000ECE1FDE02083318320E030E000501046D5
:1084F0002F4F3F4FF801322F3BBF069000E00BBFDC
:108500000092250DAA2309F05DD00091250D0023CE
:1085100009F029CF00E06EDD26CFADDC0093260DFB
:108520000091260D0093270DECE1FDE00081118103
:1085300098012F5F3F4FECE1FDE02083318320E085
:1085400030E0005010462F4F3F4FF801322F3BBF15
:10855000069000E00BBF0092250DAA2309F032D04F
:108560000091250D002309F0FECE0091270D42DD7C
:10857000AA2309F4F8CE0091270D002309F4F3CEC5
:1085800021D0F1CEAA2309F01DD00091270D0023A0
:1085900011F401E001C000E02DDDAA2309F4E3CECF
:1085A0000091270D002309F0DECE0CD0DCCE00E1D7
:1085B00010E093DED8CE0091E80C0023E1F7E3E071
:1085C0000C94E14E0CE810E00E945B4C66D00DE28A
:1085D0000E94E60D0091230D0E94CF0D0AE30E9438
:1085E000E60D00E20E94E60D0091260D0E94CF0DDF
:1085F0000DE30E94E60D08E20E94E60DEEE1FDE0CB
:10860000008111810E94ED0E0CE20E94E60D00E255
:108610000E94E60D0091240D0E94CF0D0CE20E94F5
:10862000E60D00E20E94E60DE0E2FDE0008111812E
:108630000E94ED0E09E20E94E60D00E20E94E60DA6
:108640000091250D0E94CF0D0BE70E94E60D0091D1
:10865000270D0E94CF0D0DE70E94E60D0BE50E944D
:10866000E60DECE1FDE0008111810E94ED0E0DE5CB
:108670000E94E60D0E94170F0093220D0091220D1B
:108680000B3151F404E615E10E945B4CECE1FDE096
:10869000008111810E94ED0E08950091230D003894
:1086A00029F40BE715E10E945B4C08950091230D1E
:1086B000013829F403E815E10E945B4C089500910C
:1086C000230D023829F40BE815E10E945B4C089554
:1086D0000091230D033829F403E915E10E945B4C56
:1086E00008950091230D013029F40BE915E10E9452
:1086F0005B4C08950091230D023029F403EA15E143
:108700000E945B4C08950091230D033029F40BEA7D
:1087100015E10E945B4C08950091230D043029F46B
:1087200003EB15E10E945B4C08950091230D053089
:1087300029F40BEB15E10E945B4C08950091230D89
:10874000063029F403EC15E10E945B4C089500917A
:10875000230D073029F40BEC15E10E945B4C0895C2
:108760000091230D0F3F21F403ED15E10E945B4CB6
:1087700008952091B60D2A3010F52091B60D30E005
:10878000220F331FF901E457F24F00831183E6EB08
:10879000FDE00081039500832091270D30E00091DA
:1087A000B60D10E0000F111FF801E457F24F2083BF
:1087B0003183E6EBFDE0008103950083089509E035
:1087C00010E08BDD08950091B60D0023E9F0E6EB93
:1087D000FDE000810A95008310E0000F111FF801F1
:1087E000E457F24F008111810093270DE6EBFDE085
:1087F00000810A95008310E0000F111FF801E45773
:10880000F24F0081118108950AE010E066DD0FEF5C
:108810001FEF08950E94CF4E00916C10002309F0C5
:10882000D3C000916909013009F094C0EFEDFDE07B
:1088300002811381012B09F45AC000E00093D60D88
:1088400000E010E0EBEDFDE00083118300E010E0BC
:10885000EDE6F0E10083118301E000936C10EFED91
:10886000FDE00081118145E050E00E942D4E10E0B6
:10887000E7EDFDE000831183E7EDFDE0808191816C
:10888000EFEDFDE00281138145E050E00E942D4EA6
:1088900010E0801B910BE9EDFDE080839183E9ED11
:1088A000FDE020813181243700E0300720F003E033
:1088B0000093E80D27C2E9EDFDE0208131812237E8
:1088C00000E0300720F007E00093E80D1BC2E9ED5F
:1088D000FDE020813181203700E0300720F00FE0FB
:1088E0000093E80D0FC20FE00093E80D0BC200915A
:1088F000D60D0370002309F005C2EFEDFDE0008105
:10890000118145E050E00E942D4E10E0E7EDFDE0C2
:1089100000831183E7EDFDE080819181EFEDFDE0C3
:108920000281138145E050E00E942D4E10E0801B33
:10893000910BE9EDFDE080839183E9EDFDE020817D
:108940003181293500E0300708F0DCC10FE70093E2
:10895000E80DD8C1EFEDFDE002811381012B09F094
:10896000D1C10091D60D0370002309F0CBC1EFED0A
:10897000FDE00081118145E050E00E942D4E10E0A5
:10898000E7EDFDE000831183E7EDFDE0808191815B
:10899000EFEDFDE00281138145E050E00E942D4E95
:1089A00010E0801B910BE9EDFDE080839183E9ED00
:1089B000FDE020813181293500E0300708F0A2C1B7
:1089C0000FE70093E80D9EC100916C10013009F093
:1089D0004AC1EFEDFDE002811381012B61F400E05B
:1089E00010E01BBD0ABD00E00093E80DA89800E070
:1089F00000936C1087C10091D60D0F71002329F4EC
:108A000000E010E01BBD0ABD7DC10091D60D0F71C5
:108A1000023009F077C1EFEDFDE00081118145E002
:108A200050E00E942D4E10E0E7EDFDE00083118341
:108A3000E7EDFDE080819181EFEDFDE002811381A2
:108A400045E050E00E942D4E10E0801B910BE9EDB7
:108A5000FDE080839183EBEDFDE000811181E9ED84
:108A6000FDE0208131810217130740F4E9EDFDE0BC
:108A700000811181EBEDFDE000831183EAE1F6E175
:108A8000A3EEBDE00D911C911197169507951695D3
:108A90000795E00FF11F049110E0EDEDFDE000837C
:108AA0001183E9EDFDE0008111810A5F1F4FE7EDC1
:108AB000FDE0208131810217130718F00FEF13E05A
:108AC00010C00AEF17E1E7EDFDE040815181E9EDCB
:108AD000FDE020813181421B530B465050400E94E3
:108AE0002D4E003024E0120710F00FEF13E01BBDF5
:108AF0000ABDADEDBDE0ED91FC911197F69720F028
:108B000003E00093E80D32C0ADEDBDE0ED91FC91C6
:108B10001197F49720F007E00093E80D27C0E9EDE6
:108B2000FDE020813181243700E0300720F003E0B0
:108B30000093E80D1BC0E9EDFDE020813181223773
:108B400000E0300720F007E00093E80D0FC0E9EDEA
:108B5000FDE020813181203700E0300720F00FE078
:108B60000093E80D03C00FE00093E80DEDE6F0E19F
:108B7000008111810F5F1F4F00831183EDE6F0E14B
:108B800020813181283601E0300758F000E010E004
:108B90001BBD0ABD0FEF0093E80D02E800936C10B7
:108BA000B1C0E9EDFDE020813181263700E03007DA
:108BB00058F000E010E01BBD0ABD0FEF0093E80D78
:108BC00001E800936C109EC0EBEDFDE00081118187
:108BD0000C531040E9EDFDE02081318102171307AD
:108BE00098F0E9EDFDE020813181253600E0300785
:108BF00058F000E010E01BBD0ABD0FEF0093E80D38
:108C000003E800936C107EC0EDEDFDE02081318122
:108C10002C3300E0300758F000E010E01BBD0ABD27
:108C20000FEF0093E80D04E800936C106BC0ADEDFE
:108C3000BDE0ED91FC911197F89708F463C0E9ED60
:108C4000FDE020813181203700E0300708F45AC070
:108C500000E010E01BBD0ABD0FEF0093E80D04E833
:108C600000936C104FC000916909023041F002E09E
:108C70000093690927E030E0A9010E94FF4DEFED64
:108C8000FDE002811381012BC1F400E010E01BBD67
:108C90000ABD00E00093E80DA89800E000936C1076
:108CA00000916909002371F100E00093690927E050
:108CB00030E0A9010E94FF4D25C00091D60D0F7133
:108CC000002301F5EFEDFDE00081118145E050E06A
:108CD0000E942D4E10E0E7EDFDE000831183E7EDEB
:108CE000FDE080819181EFEDFDE00281138145E09F
:108CF00050E00E942D4E10E0801B910BE9EDFDE04D
:108D000080839183E4E00C94E04E07EE06B900E026
:108D100010E01BBD0ABD03EC0FBD02E00EBD03E079
:108D20000093E70DE7EEFDE00081039500830370FB
:108D300007B901E010E00E94670C24B135B1009141
:108D4000E70D10E003701070000F111FF801E152E1
:108D5000F24F20833183E7EEFDE00081039500832D
:108D6000037007B901E010E00E94670C24B135B12F
:108D70000091E70D10E003701070000F111FF80153
:108D8000E152F24F20833183E7EEFDE0008103954D
:108D90000083037007B901E010E00E94670C24B162
:108DA00035B10091E70D10E003701070000F111F36
:108DB000F801E152F24F20833183E7EEFDE00081BC
:108DC00003950083037007B901E010E00E94670C6F
:108DD00024B135B10091E70D10E003701070000F61
:108DE000111FF801E152F24F2083318308950E9450
:108DF000D04E1A981B9A0E94E30BA89800E00093AB
:108E000070090093710900E00093720900937309DF
:108E100000E00093E80C00E00093F90C22E030E061
:108E2000A9010E94F34D0F3FA9F021E030E0A90114
:108E30000E94F34D0F3F71F023EF3FE0A9010E9424
:108E4000F34D033038F427E030E0A9010E94F34DE0
:108E5000033048F101E00093630921E030E0A9010B
:108E60000E94FF4D02E20093620920E030E0A90178
:108E70000E94FF4D00E022E030E0A9010E94FF4D7A
:108E800080E023EF3FE0082FA9010E94FF4D0AE098
:108E90000093F90C00E00093690927E030E0A90194
:108EA0000E94FF4D37C021E030E0A9010E94F34D40
:108EB0000093630920E030E0A9010E94F34D009384
:108EC000620923EF3FE0A9010E94F34D802F23E0C8
:108ED00030E0A9010E94F34D0093650924E030E0E1
:108EE000A9010E94F34D0093660929E030E0A90131
:108EF0000E94F34D00936B092AE030E0A9010E9423
:108F0000F34D00936C0927E030E0A9010E94F34D76
:108F10000093690900E000936A0911E020E830E05D
:108F200000E00E94C40B21E01091620900E00E9461
:108F3000330C21E012E201E00E94330C00E00093C8
:108F4000700900937109E1DE789424EF3FE0A901F4
:108F50000E94F34D053519F400E0C8D45EC183309A
:108F600038F080E023EF3FE0082FA9010E94FF4D79
:108F700094B700E004BF21EF3FE0A9010E94F34D48
:108F8000002361F0923051F48395833008F080E043
:108F900023EF3FE0082FA9010E94FF4D9A7099230B
:108FA00061F400916909002341F000E00093690930
:108FB00027E030E0A9010E94FF4D21EF3FE0A90129
:108FC0000E94F34D013031F001E021EF3FE0A901B3
:108FD0000E94FF4D00916909023009F05DC000E870
:108FE00000936C100FEF0093E80D56C090E0809B4B
:108FF00004C002E310E00E94670C0091090D10917B
:10900000080D011769F00E94170FA02FA53521F454
:109010000091080D0093090D082F0E94E60D01C074
:10902000A0E0882311F4AC9807C0813011F4AD980A
:1090300003C0823009F4AE98933209F046C0A332DF
:1090400009F043C004E110E00E94670C08E001BD94
:10905000809B04C002E310E00E94670C0C991CC0C6
:1090600002E310E00E94670C00916909002371F48B
:10907000EFEDFDE002811381012B41F001E000934F
:10908000690927E030E0A9010E94FF4D0C9BFECF4B
:1090900002E310E00E94670C809B31C0AD9AAC9A4D
:1090A000AE9A0091090D1091080D011709F49ECF99
:1090B0000E94170F902F953521F40091080D009311
:1090C000090D082F0E94E60D92CF993011F0A930BA
:1090D00089F404E110E00E94670C08E001BD83956B
:1090E000833008F080E023EF3FE0082FA9010E94C1
:1090F000FF4DAECF9D3019F0AD3009F0A9CF21EF73
:109100003FE0A9010E94F34D002331F000E021EF80
:109110003FE0A9010E94FF4D809BFECF04E110E0DB
:109120000E94670C00E910E0C6D38ED3882391F427
:1091300001E0DCD3902F0CE810E0BDD3092F0E9492
:109140002B0F08E512E0B7D301E0009372090E94EB
:109150003B0FFDCF00916209013059F101E000930E
:1091600062092091620914E00EEF0AD505E912E0C8
:10917000A2D300E814E82EE130E04091620950E00B
:1091800060E070E04F5F5F4F6F4F7F4F0E949C4EDB
:109190000E940E0E00EB12E08ED30091620920E0D7
:1091A00030E0A9010E94FF4D09B904EF11E00E94CF
:1091B000670C01E010E0E3EEFCE00083118301E0C6
:1091C00095D3902F0CE810E076D3092F0E942B0F37
:1091D00008E512E070D307E0009372090E94FB21BA
:1091E000EFEDFDE020813181273302E0300730F0E0
:1091F00023E333E012E20EEFCBD405C02FEF33E0D0
:1092000012E20EEFC5D4813071F401E010E0E3EE1C
:10921000FCE0008311830E94182303E0009372098D
:109220000E94992416C08230A1F404E610E00E9446
:10923000670C02E00093720900E00E94924104E68C
:1092400010E00E94670C04E110E00E94670C08E047
:1092500001BDFFCFFA93EA934A933A932A931A9364
:109260000A933FB74BB700E00BBFAA9820919C0030
:109270000091080D10E00F701070F801E65FF24FDA
:109280002083E8E0FDE00081039500834BBF3FBFF2
:1092900009911991299139914991E991F99118957B
:1092A000FA93EA934A933A932A931A930A933FB70D
:1092B0004BB700E00BBF00917009102F139510936E
:1092C00070092CB110E0F801E056F94F20834BBF34
:1092D0003FBF09911991299139914991E991F991EA
:1092E00018952497AA98A99808EA10E0E4D223C018
:1092F0000E94170F0E94E20D5E9A0091090D1091D5
:10930000080D0117A9F75E9BFECF1A981B9A0091D2
:10931000710910917009011771F00091710910E045
:10932000F801E056F94F0081E1E7F9E0108113956B
:1093300010830E94E60D0091090D1091080D011790
:1093400031F31B981A9AD9CF0E94CC4EAA98A998AB
:1093500008EA10E0B0D218C05E9BFECF1A981B9AA4
:109360000091710910917009011771F00091710954
:1093700010E0F801E056F94F0081E1E7F9E01081D3
:10938000139510830E94E60D0091090D1091080DB0
:10939000011731F31B981A9A1CC0FC013A2F3BBFEE
:1093A0000690002D10E01BBF8F5F9F4FAF4FBF4F48
:1093B000600E0E94E20D5E9A01E0400E00E0501E39
:1093C0000FEF401607E1500640F3062D0E94E20D14
:1093D0005E9A0091090D1091080D011709F4BCCF98
:1093E0000E94170F0E3741F480E090ECA0E0B0E04F
:1093F000662444245524E4CF0E94E20D5E9AE9CF0E
:109400000E94CE4E902F44249F3F29F400E014EF99
:1094100021E030E004C008EE13E020E030E080E01E
:1094200013C04091710950E0FA01E056F94F4081B4
:10943000E1E7F9E0508153955083682F70E0FB011C
:10944000EE5DF74F408383958917D8F440E050E0F4
:1094500060E070E00090710910907009011479F4D7
:109460000A011B01A001B1014F5F5F4F6F4F7F4F9A
:10947000001511052205330568F744244394442060
:1094800081F2A82FB0E00091D8080E3F09F470C017
:10949000442071F09F3F61F0E2E7F9E0008100FFB6
:1094A00003C00FE11DE007D200917009009371091C
:1094B000A43008F45DC0009122080F3F21F4009110
:1094C00023080F3F71F0E2E7F9E0008100FF03C0DD
:1094D00004E31DE0F0D1009170090093710900E0F0
:1094E00048C0009124081091D808011771F0E2E7F4
:1094F000F9E0008100FF03C00AE41DE0DCD1009127
:1095000070090093710900E034C02091250830E013
:109510000A2F10E0045010402017310771F0E2E7E5
:10952000F9E0008100FF03C000E61DE0C4D1009116
:1095300070090093710900E01CC082E007C090E050
:10954000FC01EE5DF74F0081B00F83958A17B8F3E9
:10955000BF3F71F0E2E7F9E0008100FF03C006E7DA
:109560001DE0A9D1009170090093710900E001C0CC
:109570000A2FE5E00C94DF4E0E94CF4E3FEF309370
:10958000D6083FEF3093D7080093D808022F0E5F1C
:109590000093D9081093DA0880E00DC090E0FC0138
:1095A000E056F84F0081A82FB0E01596FD01EA5271
:1095B000F74F00838395821788F300E02A5FA22F7C
:1095C00082E007C090E0FC01EA52F74F1081010FE2
:1095D000839590E0EA2FF0E031978E179F0794F380
:1095E000009590E0FC01EA52F74F00831B981A9A0D
:1095F00080E009C05E9A90E0FC01EA52F74F0081DA
:109600000E94E20D83958A17A8F35E9BFECF1A98FD
:109610001B9A0A2FE4E00C94E04E0E94CF4ED80132
:10962000922F992359F40091D8080E3F21F400EFAE
:1096300011E041D103C001E112E03DD180E00CC056
:10964000082F10E0FD01E00FF11F00810E949E0E27
:1096500000E20E94E60D8395891790F301E412E081
:109660002AD1092F0E942B0FE4E00C94E04E0E94B7
:10967000CD4E802F912F422E01E00093E70CB0E0F9
:109680002DC040E050E060E070E0F0E08A019B0116
:10969000A801B9014F5F5F4F6F4F7F4F083EE3E076
:1096A0001E07E0E02E07E0E03E0798F40091710904
:1096B00010917009011751F300917009009371091D
:1096C00040E050E060E070E00F2FF02FF39505369A
:1096D000E8F20091700900937109B395B23008F077
:1096E00051C00091700900937109242D192F082F82
:1096F00043DFA02F913061F48E3F29F455245A9412
:109700005092740930C006E0502E509274092BC05C
:10971000923039F45090A10706E0500E509274092F
:1097200022C08E3FC1F08F3140F4082F10E0F801C5
:10973000EB58F64F0081023870F0843680F08E3698
:1097400070F4082F10E004561040F801EB56F64F65
:109750000081023820F455245092740913C006E0A9
:10976000502E50927409552009F4B7CF052D48DECC
:109770000093740900917409051521F00FEF50163C
:1097800009F07FCF00E00093E70C00917409051504
:1097900009F443C00091D8080E3FF9F1E2E7F9E07F
:1097A000008100FF15C00DED1DE085D0082F0E943F
:1097B0002B0F07EB10E07FD02A2F06ED18E02DDFEE
:1097C00009EC10E078D02091740902E218E025DF5E
:1097D000E2E7F9E0008101FF1EC000E011E80E940D
:1097E0006D41082F0E949E0E00E20E94E60D092F97
:1097F0000E949E0E00E20E94E60D0091A0070E94CA
:109800009E0E00E20E94E60D0091A1070E949E0EAE
:1098100000E20E94E60D00E014C0009173090023ED
:1098200079F007EB10E047D02A2F06ED18E0F5DEBF
:1098300009EC10E040D02091740902E218E0EDDE5E
:1098400001E0E6E00C94DE4E0BED10E034D000E8D1
:1098500014E82EE130E04091990050E060E070E0C3
:109860004F5F5F4F6F4F7F4F0E949C4E0E940E0EC6
:1098700000E20E94E60D00EB12E01DD00CE20E9417
:10988000E60D05EE10E017D000E814E82EE130E018
:1098900049B150E060E070E04F5F5F4F6F4F7F4F26
:1098A0000E949C4E0E940E0E00E20E94E60D00EB0C
:1098B00012E001D00895EF97EF97A49720E001C040
:1098C0002395203A60F430E0F801E20FF31F449151
:1098D000FE0130E0E20FF31F4083442389F78E013D
:1098E0000E940A0FEF96EF96A49608950E94CF4E1D
:1098F000A02FAA2361F00CE810E0DDDF09E40E944C
:10990000E60D04E40E94E60D0AE30E94E60D90E0F5
:1099100080E00EC0843658F08E3648F420E0082FE0
:1099200010E004561040F801EB56F64F2083839563
:10993000803888F520E011E0082F99DE002309F136
:109940008F3140F420E8082F10E0F801EB58F64F73
:1099500020830DC0843658F08E3648F420E8082F56
:1099600010E004561040F801EB56F64F2083AA236E
:1099700031F0082F0E949E0E00E20E94E60D9395A2
:10998000D6CF8F3138F620E0082F10E0F801EB58E1
:10999000F64F2083CCCF40EC50EE60E070E080E0EA
:1099A00059C002E0809F8001212F220F220B322F0D
:1099B000040F151F261F371F0F5F1F4F2F4F3F4FDD
:1099C000F801322F3BBF0690102D00E00BBF00E0E6
:1099D00022E0829F212C220C2208322C040E151E1C
:1099E000261E371EF001322D3BBF069020E02BBF14
:1099F0001124000E111E082F10E0000F111FF80196
:109A0000E056F64F00821182082F10E0000F111F60
:109A1000F801E056F64F20813181203000E4300714
:109A200069F0082F10E0000F111FF801E056F64F03
:109A300020813181203000E4300759F400E010E04B
:109A4000282F30E0220F331FF901E056F64F008334
:109A5000118383958F3108F4A4CF80E012C014E203
:109A6000082F0E94BB2F0060106222E0829F20E03E
:109A7000020E22E0121EF001E052F64F0083118325
:109A800083958F3180F5082F10E0F801EB58F64FE1
:109A900000810023A9F310E1082F4DD00068282F82
:109AA00030E0F901EB58F64F008315E0082F43D062
:109AB000002321F020E015E0082F62D018E1082FE4
:109AC0003AD0013061F61EE1082F0E94BB2F22E040
:109AD000829F20E0020E22E0121EF001E052F64FBB
:109AE00000831183CDCF84E620C0A82FB0E0A45618
:109AF000B040FD01EB56F64F00810023A9F010E1C4
:109B0000082F19D00068A82FB0E0A456B040FD017E
:109B1000EB56F64F008315E0082F0DD0002321F0FF
:109B200020E015E0082F2CD083958E36F0F2092F17
:109B3000E4E00C94E04E1093A00711E01093A1070D
:109B400022E012E094DD002319F000912708089527
:109B50000FEF08951093A00712E01093A10722E0E1
:109B600012E085DD002349F03091280820E00091C3
:109B7000270810E0020F131F08950FEF1FEF08953D
:109B80001093A0072093A10722E013E070DD089551
:109B90001093A007122F1093A107232F30E02093DA
:109BA000A20723E013E063DD08950FE30DBF05E096
:109BB0000EBFC0E0D5E00E94EB4E002311F00E94E2
:109BC000FD4E00E00BBF0E94F7460E94204F0C9410
:109BD000204FE199FECF08954F5F5F4FFADF4EBBF4
:109BE0005FBBE09A0895FADF0DB308954F5F5F4FB2
:109BF0004EBB5FBBF894E29AE19A0FBE08950FB690
:109C0000E8DF0DBBF5CF0024E8E0EA9532F0001F55
:109C1000001C0416D0F3041AF8CF001F402D009545
:109C20000895002411240030010741F0169507958E
:109C300010F4040E151E440F551FF5CF002D112DE5
:109C400008954A951AF0000F111FFBCF08954A9509
:109C50001AF016950795FBCF089500241124EFE024
:109C6000001F111F001C111C0416150610F0041A09
:109C7000150AEA95AAF7001F111F402D512D0095D6
:109C80001095089530952095109501951F4F2F4FF1
:109C90003F4F089570956095509541955F4F6F4F78
:109CA0007F4F08950024112422243324E02FE12B38
:109CB000E22BE32B71F0369527951795079520F445
:109CC000040E151E261E371E440F551F661F771FD4
:109CD000EDCF002D112D222D332D08954A952AF018
:109CE000000F111F221F331FF9CF089500241124E4
:109CF00022243324E0E2EA9592F0001F111F221F74
:109D0000331F001C111C221C331C041615062606CA
:109D1000370688F3041A150A260A370AECCF001F03
:109D2000111F221F331F402D512D622D732D0095C1
:109D30001095209530950895FF2777231AF4F16048
:109D40000E944A4E33231AF4F0950E94424E0E941C
:109D5000764EF69510F40E94424EF69510F40C944F
:109D60004A4E0895AF93BF93B12FA02F3BBFD89514
:109D7000EF5FFF4F3F4F0D9241505040B9F74BBF3F
:109D8000BF91AF910895FA92EA92DA92CA92BA928A
:109D9000AA929A928A927A926A925A924A92BA9322
:109DA000AA939A938A930895FF84EE84DD84CC84E9
:109DB000BB84AA84998488847F806E805D804C8077
:109DC000BB81AA8199818881F0E00FB6F894CE0F0B
:109DD000DF1F0FBE089501E0089520E002D0E9F7EB
:109DE00008952D9301501040202F212B08953BBF43
:109DF00027913BB7F6DFD9F7089501E91EE928015D
:109E0000F20130E03BBF07911691F2013296A79123
:109E1000B691F2013496479157916691242F252BE4
:109E2000262B21F0FA01362FE2DF01C0D6DF07E052
:109E3000400E00E0501EA2014F395E4908F308951C
:109E400000008895FECF141A1F24292E33383D4D6B
:109E5000151B20252A2F3439080808090909090982
:109E60000909090909090909090909090808080866
:109E700008080808080808070700FF030205040788
:109E80000609080B0A0D0C0F0E111013121514FF02
:109E900000600140059F9E00CF09A0060000004918
:109EA000440050494E47004700474F004452455335
:109EB0004554005245534554005359535F5752007F
:109EC00041435400414354494F4E005245475F5768
:109ED0005200570057520057524954450053594EAB
:109EE000435F5752005357520043414C550044457D
:109EF00043004845580043414C430043414C440013
:109F000052000D0A205B4349443A005D200052454F
:109F1000540052455455524E0052554E0048454C3F
:109F200050004C004C544F5353005400544F535363
:109F30000043494400544553540043484B004445B2
:109F40004D4F004D4F4E49544F5200424155440031
:109F5000534541524348004C4544005343414E0051
:109F600055504441544500440044554D50004F461F
:109F700046004F4E004E414D4500434F5059005052
:109F800000504147450042004245464F5245004E71
:109F9000004E45585400474F544F004D4F4E00520D
:109FA000450053504545440054494D450052440036
:109FB0005245414400480045584954005341560019
:109FC00053415645004E4557004D004D4952524FA2
:109FD000520053455400504C4159004900494E53DA
:109FE0004552540044454C455445004D4F5645009C
:0F9FF0005300535445500042414C414E434500ED
:00000001FF
